:100000000C9463000C948B000C948B000C948B006C
:100010000C948B000C94E91D0C948B000C948B00B9
:100020000C948B000C948B000C948B000C948B0024
:100030000C948B000C948B000C948B000C948B0014
:100040000C94801C0C948B000C944E1C0C94281C5B
:100050000C948B000C948B000C948B000C948B00F4
:100060000C94CA1C0C948B00000000002400270094
:100070002A0000000000250028002B0000000000DE
:1000800023002600290004040404040404040202DA
:100090000202020203030303030301020408102007
:1000A0004080010204081020010204081020000012
:1000B0000008000201000003040700000000000027
:1000C0000000641EFE3011241FBECFEFD8E0DEBF5B
:1000D000CDBF26E0A0E8B4E001C01D92AA3EB20761
:1000E000E1F714E0A0E0B1E0E2E6F0E702C005903D
:1000F0000D92A038B107D9F710E0C2E6D0E004C0F5
:100100002197FE010E942336C136D107C9F70E940C
:100110004E1F0C9424380C940000982F2091A105B8
:1001200081E0213208F043C080917D058111FCCF30
:100130008091A00532E030937D0590937C059FEF80
:1001400090937B0510927A0520937905A0E8B5E09D
:10015000E9E5F5E090E0291331C01092580590913F
:100160005805880F892B8093580580915705813059
:1001700049F510925705809158058093BB008091F6
:10018000BC0083FDF8CF85EC8093BC0080917D0599
:100190008230E1F380917B058F3FB1F080917B0548
:1001A0008032A1F080917B05803391F084E0109241
:1001B0007F051092A10510927E0508953D9131931F
:1001C0009F5FC9CF85EEE0CF80E0F1CF82E0EFCF37
:1001D00083E0EDCF8091350590913605891B990B11
:1001E0000895089508952F923F924F925F926F92D3
:1001F0007F928F929F92AF92BF92CF92DF92EF92B7
:10020000FF920F931F93CF93DF93CDB7DEB76C9719
:100210000FB6F894DEBF0FBECDBF522E3D874E877E
:10022000252E462E372E782E692EA982BF86C88AA3
:10023000D98AEA8AFB8A0C8B1D8B988E8F8A2115AE
:1002400000EA30070CEA400709EB500703E06007BB
:1002500071058105910509F098F52F3F10EE3107E2
:1002600015EF410715E051076105710581059105FD
:1002700009F008F40BC12F3F354D41415E47634003
:1002800071058105910509F008F40BC129813F85AD
:10029000488959896A897B898C899D89A0E099243C
:1002A00093940E940336C9F4F1E0FE8B04E0802EA3
:1002B000912CA12CB12C89869A86AB86BC8616C15E
:1002C000512CB0EABD87ECEAEE8789EB282E93E04B
:1002D000492E312C712C612CD9CFA52CBD84CE8414
:1002E000D22CE42CF32C072D162D29813F8548892B
:1002F00059896A897B898C899D890E944E35298715
:100300003A874B875C8729853A854B855C85B6E0C3
:10031000AB2EB12C263031054105510568F0898599
:100320009A85AB85BC8589309740A105B105E0F081
:10033000F8E0AF2EA7E0BA2EC12CD12CE12CF12C85
:1003400000E010E029813F85488959896A897B89C5
:100350008C899D890E944E35522E3D874E87252ED1
:10036000462E372E782E692EA52CBD84CE84D22C15
:10037000E42CF32C072D162D29813F8548895989B6
:100380006A897B898C899D890E944C35AA24AA940C
:10039000BB24BA94EFE0CE2ED12CE12CF12C00E05E
:1003A00010E00E948934A52CBD84CE84D22CE42C8C
:1003B000F32C072D162D0E944E35A32FF42FE52F79
:1003C000422F5A2F6F2F7E2FCC24CA94DC2C8FE023
:1003D000E82EF12C411551056105710521F4C12C60
:1003E000D12C7601C394AA24A3949A1409F4E5C0ED
:1003F00001E00E8BCB01BA0137E0660F771F881F33
:10040000991F3A95D1F7A70196010E944834298F88
:100410003A8F4B8F5C8F89849A84AB84BC8447E08D
:10042000880C991CAA1CBB1C4A95D1F79501840124
:1004300012502109310948015901298D3A8D4B8DFE
:100440005C8D280D391D4A1D5B1DAF89B88D2D931C
:100450003D934D935C931397FD016483758386836D
:1004600097831896CD92DD92ED92FC921B978E8821
:10047000882009F481C059829D849F86AE84A88A11
:10048000298A4A8A3B8A7C8A6D8A76C0512C01EE81
:100490000D8715EF1E8725E0222E412C312C712C63
:1004A000612C29813F85488959896A897B898C8992
:1004B0009D89A0E0912C0E94033609F00ECFA52C57
:1004C000BD84CE84D22CE42CF32C072D162D20E0F5
:1004D00034E04BE654EF64E170E080E090E00E948D
:1004E0004E3529873A874B875C871E8A89849A8490
:1004F000AB84BC84A501940160E070E0CB01A52C25
:10050000BD84CE84D22CE42CF32C072D162D298308
:100510003A834B835C836D837E838F83988760E00F
:1005200070E080E090E00E94893429833F87488B07
:10053000598B6A8B7B8B8C8B9D8B0E89C12CD12C1C
:100540007601C39440E050E0BA01013009F052CF87
:10055000AF89B88D1D921D921D921C921397FD01BB
:10056000148215821682178281E090E0A0E0B0E04C
:1005700080879187A287B38729813F8548895989D8
:100580006A897B898C899D896C960FB6F894DEBF49
:100590000FBECDBFDF91CF911F910F91FF90EF90D4
:1005A000DF90CF90BF90AF909F908F907F906F9093
:1005B0005F904F903F902F900895AF89B88D1D9216
:1005C0001D921D921C921397FD01148215821682B2
:1005D000178281E090E0A0E0B0E080879187A28759
:1005E000B3875982FD85FF878E84888A49CFDF9241
:1005F000EF92FF920F931F93CF93DF93FC01E08064
:10060000F18002811381D481C581B681D7809701A1
:10061000A8016D2F7C2F8B2F9D2D35534C405109F8
:1006200061097109810991092F3F34434C405105FB
:10063000610571058105910509F0D0F49701A801C4
:100640006D2F7C2F8B2F9D2D07E00E94BB352083C3
:10065000318342835383648375838683978387E0E2
:10066000DF91CF911F910F91FF90EF90DF90089550
:100670009701A8016D2F7C2F8B2F9D2D3A56484155
:10068000510961097109810991092F3F3946484192
:100690005105610571058105910509F098F49701EF
:1006A000A8016D2F7C2F8B2F9D2D06E00E94BB355E
:1006B0002083318342835383648375838683978346
:1006C00086E0CECF9701A8016D2F7C2F8B2F9D2D1B
:1006D000345D4043510961097109810991092F3F36
:1006E000334D40435105610571058105910509F0C0
:1006F00098F49701A8016D2F7C2F8B2F9D2D05E07D
:100700000E94BB3520833183428353836483758386
:100710008683978385E0A4CF9701A8016D2F7C2F56
:100720008B2F9D2D385A4146510961097109810964
:1007300091092F3F374A41465105610571058105F1
:10074000910509F098F49701A8016D2F7C2F8B2F4C
:100750009D2D04E00E94BB35208331834283538367
:10076000648375838683978384E07ACF9701A80199
:100770006D2F7C2F8B2F9D2D3055434C51096109D6
:100780007109810991092F3F3F44434C510561058F
:1007900071058105910509F098F49701A8016D2F65
:1007A0007C2F8B2F9D2D03E00E94BB35208331834E
:1007B00042835383648375838683978383E050CF1A
:1007C0009701A8016D2F7C2F8B2F9D2D305A464805
:1007D000514061097109810991092F3F3F494648FC
:1007E0005140610571058105910509F098F4970163
:1007F000A8016D2F7C2F8B2F9D2D02E00E94BB3511
:1008000020833183428353836483758386839783F4
:1008100082E026CF9701A8016D2F7C2F8B2F9D2D75
:1008200030544D40534061097109810991092F3FAE
:100830003F434D405340610571058105910509F025
:1008400098F49701A8016D2F7C2F8B2F9D2D01E02F
:100850000E94BB3520833183428353836483758335
:100860008683978381E0FCCE80E0FACE0895DB0199
:1008700014964D915C9115976D917C91DC01ED91F1
:10088000FC910280F381E02D0994AF92BF92CF9248
:10089000DF92EF92FF920F931F93CF93DF936C0140
:1008A0007B018B01040F151FEB015E01AE18BF0821
:1008B000C017D10759F06991D601ED91FC910190D3
:1008C000F081E02DC6010995892B79F7C501DF91EB
:1008D000CF911F910F91FF90EF90DF90CF90BF903D
:1008E000AF900895FC01538D448D252F30E0842F67
:1008F00090E0821B930B541710F0CF960895019748
:100900000895FC01918D828D981761F0A28DAE0F34
:10091000BF2FB11D5D968C91928D9F5F9F73928FBB
:1009200090E008958FEF9FEF0895FC01918D828DE7
:10093000981731F0828DE80FF11D858D90E00895B4
:100940008FEF9FEF0895FC01918D228D892F90E00C
:10095000805C9F4F821B91098F739927089582EACB
:1009600095E00E94A30421E0892B09F420E0822F66
:10097000089580E090E0892B29F00E94AF04811156
:100980000C9400000895FC01A48DA80FB92FB11D8F
:10099000A35ABF4F2C91848D90E001968F739927B5
:1009A000848FA689B7892C93A089B1898C91837093
:1009B00080648C93938D848D981306C00288F3898C
:1009C000E02D80818F7D80830895EF92FF920F93B9
:1009D0001F93CF93DF93EC0181E0888F9B8D8C8DEB
:1009E00098131AC0E889F989808185FF15C09FB7DF
:1009F000F894EE89FF896083E889F98980818370A2
:100A0000806480839FBF81E090E0DF91CF911F9150
:100A10000F91FF90EF900895F62E0B8D10E00F5F71
:100A20001F4F0F731127E02E8C8D8E110CC00FB647
:100A300007FCFACFE889F989808185FFF5CFCE01DF
:100A40000E94C304F1CFEB8DEC0FFD2FF11DE35A93
:100A5000FF4FF0829FB7F8940B8FEA89FB89808162
:100A60008062CFCFCF93DF93EC01888D8823B9F0DC
:100A7000AA89BB89E889F9898C9185FD03C08081A9
:100A800086FD0DC00FB607FCF7CF8C9185FFF2CF26
:100A9000808185FFEDCFCE010E94C304E9CFDF91B5
:100AA000CF910895833081F028F4813099F082301D
:100AB000A9F008958730A9F08830C9F08430B1F4E6
:100AC000809180008F7D03C0809180008F7780931C
:100AD0008000089584B58F7784BD089584B58F7D97
:100AE000FBCF8091B0008F778093B0000895809104
:100AF000B0008F7DF9CFCF93DF93282F30E0F9013D
:100B0000E255FF4F8491F901E656FF4FD491F90168
:100B1000EA57FF4FC491CC23A1F081110E945205E6
:100B2000EC2FF0E0EE0FFF1FE458FF4FA591B491BA
:100B3000EC91ED2381E090E009F480E0DF91CF912A
:100B4000089580E090E0FACF1F93CF93DF93282F92
:100B500030E0F901E255FF4F8491F901E656FF4F6D
:100B6000D491F901EA57FF4FC491CC23A9F0162F75
:100B700081110E945205EC2FF0E0EE0FFF1FEE589E
:100B8000FF4FA591B4918FB7F894EC91111108C063
:100B9000D095DE23DC938FBFDF91CF911F91089515
:100BA000DE2BF8CF109236051092350510927F0596
:100BB0001092A10510927D0581E080937C05109232
:100BC000570561E082E10E94A40561E083E10E9493
:100BD000A405E9EBF0E080818E7F808380818D7FAA
:100BE000808388E48093B80085E48093BC0081EF23
:100BF00090E0909334058093330582EF90E09093DA
:100C00003205809331050895CF93DF9390E0FC0186
:100C1000E656FF4F24918A579F4FFC018491882309
:100C2000C9F090E0880F991FFC01E859FF4FA5918A
:100C3000B491FC01EE58FF4FC591D49161110DC0E4
:100C40009FB7F8948C91209582238C9388812823D8
:100C500028839FBFDF91CF910895623051F49FB7F1
:100C6000F8943C91822F809583238C93E8812E2BDE
:100C7000EFCF8FB7F894EC912E2B2C938FBFEACF48
:100C80008E50806480937C0080917A008064809391
:100C90007A0080917A0086FDFCCF80917800909157
:100CA000790008953FB7F8948091D1049091D204CF
:100CB000A091D304B091D40426B5A89B05C02F3FC2
:100CC00019F00196A11DB11D3FBFBA2FA92F982F72
:100CD0008827BC01CD01620F711D811D911D42E06D
:100CE000660F771F881F991F4A95D1F708958F9235
:100CF0009F92AF92BF92CF92DF92EF92FF924B0101
:100D00005C010E9452066B017C010E9452066C1924
:100D10007D098E099F09683E734081059105A8F3FE
:100D200021E0821A9108A108B10888EEC80E83E07C
:100D3000D81EE11CF11C81149104A104B10429F70F
:100D4000FF90EF90DF90CF90BF90AF909F908F90EB
:100D500008952FB7F8946091CD047091CE048091DE
:100D6000CF049091D0042FBF089585ED8093BC00EF
:100D70008091BC0084FDFCCF10927D0508952091E8
:100D8000A904260F3327331F21323105ECF42091BB
:100D90007D05FC0190E080E0243069F082E0089558
:100DA000A091A9042191AC0147575B4FA40FB52F27
:100DB000B11D2C930196861798F38091A904680FB2
:100DC0006093A90480E0089581E008950895E0917A
:100DD000360580913505E81730F4F0E0E95CFA4F0C
:100DE000808190E008958FEF9FEF089590913605F0
:100DF000809135052FEF3FEF981748F4E92FF0E089
:100E0000E95CFA4F208130E09F5F90933605C9017D
:100E10000895CF92DF92EF92FF920F931F93CF939B
:100E2000DF937C01CB018A0120917E05222389F08A
:100E3000EB016B01C40ED51ECC15DD0569F069917F
:100E4000D701ED91FC910190F081E02DC70109954A
:100E5000F3CF642F0E94BF06C801DF91CF911F918D
:100E60000F91FF90EF90DF90CF900895CF93DF9395
:100E70001F92CDB7DEB7698320917E052223F9F05A
:100E80002091A105203258F021E030E0FC013383AD
:100E9000228390E080E00F90DF91CF9108958091C0
:100EA0007F05E82FF0E0E058FA4F998190838F5F3B
:100EB00080937F058093A10581E090E0ECCF61E015
:100EC000CE0101960E94BF06F7CFCF93C62F91E0C7
:100ED00090937E0590E69093A00510927F05109266
:100EE000A105682F8FE396E00E9436076C2F8FE3F1
:100EF00096E00E94360781E0CF910C948D000F930D
:100F00001F93CF93DF938B0191E090937E0590E642
:100F10009093A00510927F051092A105682F8FE392
:100F200096E00E943607E801085F1F4F69918FE342
:100F300096E00E943607C017D107C1F781E0DF9124
:100F4000CF911F910F910C948D0090E080E0089557
:100F50008FE00E9440069093FE048093FD04BC0144
:100F6000990F880B990B0E94883120E030E040EA0D
:100F700050E40E94E73120E030E040E85AE30E946C
:100F8000E73160938504709386048093870490937F
:100F9000880408958091E3049091E40440E95AE3C1
:100FA0006CE170E0009739F08130910561F540ED1A
:100FB00051EB67E370E040938301509384016093A9
:100FC0008501709386011092EF041092F004109244
:100FD000F1041092F2048530910561F580E49DE7FB
:100FE000A4E1B1E08093830190938401A0938501F3
:100FF000B09386011092EF041092F0041092F10465
:101000001092F204089582309105E1F440E153E931
:101010006BE670E0409383015093840160938501F7
:10102000709386011092EF041092F0041092F10474
:101030001092F20486309105E1F480ED9FE3A4E480
:10104000B1E0D0CF83309105E1F440E45BE66AE99A
:1010500070E0409383015093840160938501709305
:1010600086011092EF041092F0041092F104109295
:10107000F2048730910529F580E99BE3AEE7B1E002
:10108000B1CF8430910509F0A6CF40E759EE67ED66
:1010900070E04093830150938401609385017093C5
:1010A00086011092EF041092F0041092F104109255
:1010B000F204099709F0A6CF80EC92E3AAE0B3E02E
:1010C00091CF88309105A9F780E290EEA2EBB1E0D4
:1010D00089CFCF93DF9391E090937E0590E6909334
:1010E000A00510927F051092A105682F8FE396E06E
:1010F0000E94360781E00E948D0080917D0581115C
:10110000FCCF81E080937D0510927C059FEF90934A
:101110007B0510927A05109279058093580580918D
:101120005805806C8093580580915705813061F592
:1011300010925705809158058093BB008091BC00A8
:1011400083FDF8CF85EC8093BC0080917D058130D4
:10115000E1F380917A05811119C080917A05E9E562
:10116000F5E0A7E3B5E0C0E0C81312C01092360561
:10117000C093350580913605C81771F08FE396E06E
:101180000E94F606D82FF6CF85EEDDCF81E0E7CFBF
:1011900091919D93CF5FE8CF8D2FDF91CF910895EF
:1011A000CF93C0E1C80F8C2F0E946908682F63603D
:1011B0008C2FCF910C946507CF93DF93D82FC62F38
:1011C00083E00E94690861E070E001C0660FDA9573
:1011D000EAF7C13039F46095682383E0DF91CF915D
:1011E0000C946507682BF9CF0F931F93CF938B0156
:1011F000C0E1C80F8C2F0E946908682F012B39F4B9
:101200006F7D8C2FCF911F910F910C9465076062B9
:10121000F8CFCF93DF93EC0160E08E810E94A405AC
:1012200061E08E810E94A40560E08E810E94A40589
:101230008BE891E00197F1F7DF91CF910895CF927C
:10124000DF92EF92FF920F931F93CF93DF936C0186
:101250007C0187E0E80EF11CD0E0C0E0062F10E032
:10126000B8010C2E02C0759567950A94E2F761707B
:10127000F70181917F010E94A4052196C430D10518
:1012800079F7C601DF91CF911F910F91FF90EF90F9
:10129000DF90CF900C940909CF92DF92EF92FF92EA
:1012A0000F931F93CF93DF93EC01F62E642F8C8165
:1012B0000E94A4058D818F3F19F060E00E94A40573
:1012C0000F2D10E08F8584FF25C06E0187E0C80ECA
:1012D000D11CF12CE12CB8010E2C02C0759567953C
:1012E0000A94E2F76170F60181916F010E94A405F2
:1012F000FFEFEF1AFF0A88E0E816F10461F7CE016C
:10130000DF91CF911F910F91FF90EF90DF90CF90E1
:101310000C940909B80184E0759567958A95E1F701
:10132000CE010E941F096F2DCE01DF91CF911F9139
:101330000F91FF90EF90DF90CF900C941F0940E049
:10134000682F8EEC96E00C944C09CF93DF9382309B
:1013500029F49091DD0698609093DD068093E10674
:101360001092E20680E48093E30680E18093E40635
:1013700080E58093E50661E08091D2060E94040634
:101380008091D3068F3F19F061E00E94040661E06E
:101390008091D4060E940406CEECD6E09E012E5C1D
:1013A00036408091DD0684FD0BC084E090E02196FC
:1013B0002817390744F461E08E810E940406EECFBD
:1013C00088E090E0F4CF8BE39DE00197F1F760E0D7
:1013D0008091D2060E94A40560E08091D4060E940C
:1013E000A4058091D3068F3F19F060E00E94A40508
:1013F0008091DD0684FD39C063E08EEC96E00E94AA
:101400001F09CBE4D6E4CE010197F1F763E08EEC3F
:1014100096E00E941F092197F1F763E08EEC96E0B9
:101420000E941F0983E592E00197F1F762E08EECDC
:1014300096E00E941F098091DD0680620E949F094C
:1014400084E08093DE068CE00E949F0981E00E9488
:101450009F098BE39FE10197F1F782E08093DF061C
:1014600086E0DF91CF910C949F0980620E949F09D2
:101470008BE496E40197F1F78091DD0680620E948B
:101480009F0983E592E00197F1F78091DD06806284
:101490000E949F09D0CF9091E106691710F06FEF7D
:1014A000690FE62FF0E0E253F94F9489890F8068C5
:1014B0000C949F0941E00E944C0981E090E008955E
:1014C0000F931F93CF93DF938B0128E0829FC0017E
:1014D000112480640E949F09E801085F1F4F6991F1
:1014E0008EEC96E00E945A0AC017D107C1F7DF912F
:1014F000CF911F910F91089541E0682F8EEC96E0F7
:101500000E944C0981E090E00895FC0101900020C8
:10151000E9F73197AF01481B590BBC018EEC96E0FF
:101520000C9445048F929F92AF92BF920F931F939A
:10153000CF93DF93CDB7DEB7A1970FB6F894DEBF98
:101540000FBECDBF19A2423008F44AE08E010F5DF4
:101550001F4F842E912CB12CA12CA50194010E9427
:101560004834E62FB901CA01EA30F4F4E05DD8014D
:10157000EE938D01232B242B252B79F790E080E02F
:10158000109719F0CD010E94850AA1960FB6F89424
:10159000DEBF0FBECDBFDF91CF911F910F91BF90E6
:1015A000AF909F908F900895E95CE1CFCF92DF924A
:1015B000EF92FF92CF93DF9397FF19C06B017C01ED
:1015C0008DE20E947C0AEC0166277727CB016C191B
:1015D0007D098E099F094AE00E94920A8C0F9D1F87
:1015E000DF91CF91FF90EF90DF90CF9008954AE088
:1015F000DF91CF91FF90EF90DF90CF900C94920A03
:10160000CF92DF92EF92FF92CF93DF9360E083E07F
:101610000E944B0A80E20E947C0A609183017091D3
:101620008401809185019091860120E432E44FE0AD
:1016300050E00E94483469017A012A30310518F4DB
:1016400080E20E947C0A4AE0C701B6010E94920A29
:101650008EE20E947C0A60918301709184018091E6
:1016600085019091860120E432E44FE050E00E9431
:10167000483428EE33E040E050E00E9448346901ED
:101680007A01E9012436310540F480E30E947C0AA6
:101690002A9718F480E30E947C0A4AE0C701B60149
:1016A0000E94920A8EE20E947C0A609183017091EE
:1016B0008401809185019091860128EE33E040E01D
:1016C00050E00E9448346B017C01EB0164367105E7
:1016D00040F480E30E947C0A2A9718F480E30E9479
:1016E0007C0A4AE0C701B6010E94920A80E20E9489
:1016F0007C0A60E08FE00E944B0A67E876E08EEC9F
:1017000096E00E94370460E080E00E944B0A61E8A6
:1017100076E08EEC96E0DF91CF91FF90EF90DF9036
:10172000CF900C9437040C94850A80910705909112
:10173000080561E0019709F451C080E00E944B0A5E
:1017400080916C0190916D01A0916E01B0916F013B
:1017500084369105A105B10591F190F48A30910587
:10176000A105B10531F182339105A105B10521F142
:101770000197A105B105C1F589ED91E00C94930B9A
:10178000883E23E09207A105B105F9F030F4843FCB
:101790009140A105B105B1F00895803127E292078B
:1017A000A105B105A9F0803A9648A140B10599F08C
:1017B00008958EED91E0E2CF83EE91E0DFCF88EEE9
:1017C00091E0DCCF8DEE91E0D9CF82EF91E0D6CFE2
:1017D00087EF91E0D3CF8CEF91E0D0CF80E00E94F3
:1017E0004B0A81E092E0CACF0895CF92DF92EF9248
:1017F000FF9261E084E00E944B0A60917E0170914B
:101800007F01809180019091810120E432E44FE0DA
:1018100050E00E946A3469017A01C0928104D0923A
:101820008204E0928304F09284048AE0C816D10412
:10183000E104F1041CF480E20E947C0AC701B601B5
:101840000E94D60A8EE20E947C0A60917E0170910D
:101850007F01809180019091810120E432E44FE08A
:1018600050E00E946A3428EE33E040E050E00E94ED
:101870006A3469017A01C0928104D0928204E092B4
:101880008304F092840484E6C816D104E104F104D0
:1018900064F480E30E947C0A8AE0C816D104E10463
:1018A000F1041CF480E30E947C0AC701B6010E9487
:1018B000D60A8EE20E947C0A60917E0170917F01BF
:1018C000809180019091810128EE33E040E050E06A
:1018D0000E946A346B017C01C0928104D092820420
:1018E000E0928304F092840484E6C816D104E104F3
:1018F000F10464F480E30E947C0A8AE0C816D104F3
:10190000E104F1041CF480E30E947C0AC701B601E3
:101910000E94D60A80EE91E0FF90EF90DF90CF908A
:101920000C94930B4F925F926F927F928F929F9243
:10193000AF92BF92CF92DF92EF92FF920F931F93DD
:10194000CF936B017C01742EAC019B010E941F346C
:10195000882399F086E092E0CF911F910F91FF903C
:10196000EF90DF90CF90BF90AF909F908F907F903F
:101970006F905F904F900C94850A46015701E89450
:10198000B7F82FEF3FEF4FE75FE7C501B4010E94C3
:101990001F3481110DC02FEF3FEF4FE75FE7C50107
:1019A000B4010E94813118161CF48AE092E0D4CF71
:1019B0002FEF3FEF4FE75FE4C701B6010E941A34F3
:1019C00018161CF48EE092E0C7CF2FEF3FEF4FE7E1
:1019D0005FECC701B6010E94813187FDF3CF20E0A3
:1019E00030E0A901C701B6010E94813110E000E09A
:1019F00087FF08C08DE20E947C0A8C01F7FAF09400
:101A0000F7F8F094C0E060E070E080E09FE37C16BF
:101A100041F020E030E040E251E40E947933CF5FB2
:101A2000F6CFA70196010E940D332B013C010E94C5
:101A3000EB334B015C014AE00E94920A7C01E00E0C
:101A4000F11ECC23B1F1C501B4010E9486319B0186
:101A5000AC01C301B2010E940C334B015C018EE268
:101A60000E947C0AE80EF91EC15018F120E030E017
:101A700040E251E4C501B4010E94E7312B013C0171
:101A80000E94EB334B01B12CA12C4AE0C501B401FB
:101A90000E94920AE80EF91EC501B4010E94863127
:101AA0009B01AC01C301B2010E940C334B015C01EC
:101AB000DBCFC701CF911F910F91FF90EF90DF9087
:101AC000CF90BF90AF909F908F907F906F905F90DE
:101AD0004F9008952F923F924F925F926F927F9214
:101AE0008F929F92AF92BF92CF92DF92EF92FF922E
:101AF0000F931F93CF93DF93CDB7DEB76A970FB6DF
:101B0000F894DEBF0FBECDBF2F8B3987488F598F1A
:101B10006A877A8F1C011E8B0D8B6091CA067091AB
:101B2000CB068091CC069091CD0624E630E040E0D3
:101B300050E00E94F034522E632E742E852E962E85
:101B4000788B8F87492E8091C4069091C506A0910D
:101B5000C606B091C7066C017D01FF0CCC08DC2CD9
:101B600076019C01AD016C2D7C2D8C2D9C2D0FE1FF
:101B70000E94BB35A12CEAECBE2EFAE9CF2EABE3D6
:101B8000DA2EE12CF12C00E010E00E941D35A52C8E
:101B9000B62CC72CD82CE92CF8880F85142D0E9460
:101BA00089340FE10E94D63529833A834B835C83C5
:101BB0006D837E838F83988789819A81AB81BC8175
:101BC000BB0F880B982FDC018B879C87AD87BE8766
:101BD000252D362D472D582D692D7F2D8F85942D40
:101BE000A980BA80CB80DC80EB84FE2C0E2D1E2DCC
:101BF0000E94F13529833B874F87588B698B7A8BFD
:101C00008B8B9C8B8F889A8C282D3985488D598D8C
:101C10006A85792DC101211534404B46544F6441EA
:101C200071058105910569F060F0812CB4E0B987F8
:101C3000EBE6E88FF4EFF98F84E18A87912C212C71
:101C4000312C282D3985488D598D6A85792DC10112
:101C5000211538454744584F6D4071058105910560
:101C600060F4812CB8E5B987E7E4E88FF8EFF98FE5
:101C70008DE08A87912C212C312CA980BB84CF84C4
:101C8000D888E988FA880B891C89282D3985488DE0
:101C9000598D6A85792DC1010E944E3529013A017D
:101CA0001FE0A12E9FE0491651046104710440F029
:101CB000ABE54A16510461047104D0F0BAE5AB2ECD
:101CC000B12CC12CD12CE12CF12C00E010E02981A9
:101CD0003B854F85588969897A898B899C890E94BF
:101CE0008934822E3987488F598F6A87972E1C0135
:101CF000A980BB84CF84D888E988FA880B891C899D
:101D0000282D3985488D598D6A85792DC1010E940C
:101D10004C35AA24AA94BB24BA94AFE0CA2ED12C85
:101D2000E12CF12C00E010E00E948934A980BB84F2
:101D3000CF84D888E988FA880B891C890E944E359F
:101D4000C901DA01812C912C540183940097A105DB
:101D5000B10531F088248A94982CEFE0AE2EB12C96
:101D6000BC01CD0127E0660F771F881F991F2A95B8
:101D7000D1F7A50194010E944834362E272E182F42
:101D800067E0440C551C661C771C6A95D1F7B2E0DD
:101D90005B1A61087108420E531E641E751E84E1B1
:101DA00090E00E9429369A838983FC019082818287
:101DB000862D83708283538244827CE0B694A794FC
:101DC000979487947A95D1F7F82DF07F8F2E812AFA
:101DD000A981BA8115968C92159716962C92169712
:101DE00017963C921797ED89FE89BD018AE1EF2B8A
:101DF00019F069817A8182E20E947F0789819A8144
:101E00006A960FB6F894DEBF0FBECDBFDF91CF91BB
:101E10001F910F91FF90EF90DF90CF90BF90AF9008
:101E20009F908F907F906F905F904F903F902F90FA
:101E30000C94C5362F923F924F925F926F927F9291
:101E40008F929F92AF92BF92CF92DF92EF92FF92CA
:101E50000F931F93CF93DF93CDB7DEB72D970FB6B8
:101E6000F894DEBF0FBECDBF3C01C982DA82EB829F
:101E7000FC820D831E832F83388749875A876B879F
:101E80007C878AA18D873C2C2D2C9E2C502E412E98
:101E9000B22EC984DA84EB84FC8484E190E00E9451
:101EA00029368C01FC01D082C182862D880F880FD3
:101EB000880F845D0E946908F92DF3709F2E8C7F36
:101EC000982AF8019282238234824CE0F694E794B7
:101ED000D794C7944A95D1F7FC2DF07FCF2E8B2D48
:101EE0008F70C82AF801C58246825782B80182E302
:101EF000F1E06F16710431F082E06816710409F4A4
:101F000047C08AE20E947F0730E1F32EF60C8F2D46
:101F10000E94690891E0682FA9123CC060648F2D6F
:101F20000E946507E1E06E167104B1F1F2E06F16F0
:101F30007104B9F1A092C1062CE2F22E8F2D0E94FD
:101F4000690883789D8591118C60E0E18E9EB001D7
:101F50001124682B8F2D0E946507C8012D960FB69E
:101F6000F894DEBF0FBECDBFDF91CF911F910F91CF
:101F7000FF90EF90DF90CF90BF90AF909F908F90A9
:101F80007F906F905F904F903F902F900C94C5364C
:101F90008AE3B8CF6F7BC3CFA092C20694E3F92E39
:101FA000CDCFA092C3068CE3F82EC8CF2F923F92DC
:101FB0004F925F926F927F928F929F92AF92BF9259
:101FC000CF92DF92EF92FF920F931F93CF93DF9305
:101FD000CDB7DEB7AA970FB6F894DEBF0FBECDBF60
:101FE000622E298F732E3A8F4B8F5C8F6D8F7E8F71
:101FF0008F8F98A319A708A793012F3F34434C4014
:102000005105610571058105910509F050F4198E9E
:1020100085E38A8F8CE08B8F1C8E1D8E1E8E1F8E0B
:1020200018A2298D3A8D4B8D5C8D6D8D7E8D8F8D97
:1020300098A12115304A4C4A594B634071058105DE
:10204000910569F060F0198E80EA8A8F8CEA8B8F97
:1020500089EB8C8F83E08D8F1E8E1F8E18A2CE0190
:1020600049960E94F7028FA3798CBA8DAB8DFC8DB7
:10207000ED8D6E8C5F8C48A0272D3B2F4A2F5F2F54
:102080006E2F762D852D942D2F3F05ED300701E124
:1020900040070EE7500703E06007710581059105D1
:1020A00011F008F09EC0CE010D964C01A12CEEE27D
:1020B000BE2EF9E5CF2EA6E7DA2EB1E1EB2EF12CFC
:1020C00000E010E0852D942D0E94F300798D6A8D3B
:1020D0005B8D4C8D3D8D2E8D9F8D88A1E8A5F9A53A
:1020E000E130F10509F445C0329709F45EC0709300
:1020F000A9066093AA065093AB064093AC063093B2
:10210000AD062093AE069093AF068093B00680E0B4
:1021100019A2412CFEE2FAA309E50BA316E71CA3C2
:1021200091E19DA3512C612C712C8F938FA0A82E2F
:10213000CD84DE84EF84F88809891A892B893C894B
:102140004D895E896F89788D88A599A50E941A0F9F
:102150000F9099A1913009F0FBC08101242D3AA183
:102160004BA15CA16DA1752DC3010E946A0D19A23E
:10217000EFC07093B1066093B2065093B3064093DC
:10218000B4063093B5062093B6069093B7068093B5
:10219000B80680E019A2412CEEE2EAA3F9E5FBA320
:1021A00006E70CA311E11DA3BDCF7093B9066093A0
:1021B000BA065093BB064093BC063093BD062093ED
:1021C000BE069093BF068093C00680E019A2412C02
:1021D0009EE29AA3E9E5EBA3F6E7FCA301E10DA3D8
:1021E000A1CFCE010D964C01A12CB12CC12CD12C2C
:1021F000E12CF12C00E010E0852D942D0E94F300DD
:10220000298C3A8CBB8DAC8DFD8DEE8D08A519A562
:102210000130110509F44EC00230110509F4A5C1C1
:1022200000E010E091014B2F5A2F6F2F7E2F8F8DE2
:1022300098A10E94F300422E3AA34BA35CA36DA386
:10224000572E3C0170E060E090E080E00E94F408CE
:10225000409299069AA190939A06EBA1E0939B066F
:10226000FCA1F0939C060DA100939D0650929E0642
:1022700060929F067092A006898D8093A9068A8D30
:102280008093AA068B8D8093AB068C8D8093AC06D1
:102290008D8D8093AD068E8D8093AE068F8D80934D
:1022A000AF0688A18093B00681E011E019A3312C1C
:1022B000212C3BCF0F8D09A318A11EA31091C90695
:1022C000123009F019C191014B2F5A2F6F2F7E2F19
:1022D000802F9EA130584A415640610971098109F9
:1022E00091092F37304E42475849624071058105A8
:1022F000910509F008F446C02091B9063091BA065C
:102300004091BB065091BC066091BD067091BE061F
:102310008091BF069091C0065101CB2EDA2EEF2E90
:10232000FE2E09A11EA10E94FA3561F11092B1069C
:102330001092B2061092B3061092B4061092B5062F
:102340001092B6061092B7061092B80611E019A3C3
:1023500089A1AA960FB6F894DEBF0FBECDBFDF915C
:10236000CF911F910F91FF90EF90DF90CF90BF9092
:10237000AF909F908F907F906F905F904F903F9025
:102380002F9008954090A1068091A2068AA3909173
:10239000A3069BA30091A4060CA31091A5061DA360
:1023A0005090A6066090A7067090A806CE010D96E4
:1023B0004C01A42CBAA0CBA0D02EE12EF52C830189
:1023C00091014B2F5A2F6F2F7E2F89A19EA10E9422
:1023D000F30061E070E081E090E00E94F40819A24F
:1023E000298D3A8D4B8D5C8D6D8D7E8D8F8D98A155
:1023F00030584A41564061097109810991092F37C6
:10240000304E42475849624071058105910509F0F7
:1024100008F4A7C081E08093C9062091B9063091E5
:10242000BA064091BB065091BC066091BD06709102
:10243000BE068091BF069091C006A0E00E940336C0
:10244000F1F189EB96E00E94F7028FA3A090A1061C
:10245000B090A206C090A306D090A406E090A50676
:10246000F090A6060091A7061091A8062091B90643
:102470003091BA064091BB065091BC066091BD06F2
:102480007091BE06CE0101964C018091BF069091DD
:10249000C0060E94F3001F928FA0A12CC980DA8091
:1024A000EB80FC800D811E812F81388549855A85FE
:1024B0006B857C8582E090E00E941A0F0F90898DD9
:1024C0008093B1068A8D8093B2068B8D8093B3067C
:1024D0008C8D8093B4068D8D8093B5068E8D809300
:1024E000B6068F8D8093B70688A18093B80681E0E9
:1024F00022242394312C19CE2093A1063093A206D6
:102500004093A3065093A4066093A5067093A60675
:102510008093A7069093A8068E01035F1F4F480182
:10252000A12CB12CC12CD12CE12CF12C00E010E01D
:1025300091014B2F5A2F6F2F7E2F89A19EA10E94B0
:10254000F300422E3AA34BA35CA36DA3572E3C018C
:1025500061E070E081E090E00E94F40811E019A3CE
:102560003FCF88E08093C906AACF0091C90609A38E
:102570001F8D1EA308A10AA719A1113009F0F9C0E7
:1025800091014B2F5A2F6F2F7E2F8EA1902F3058F5
:102590004A41564061097109810991092F37304E2E
:1025A00042475849624071058105910561F158F132
:1025B0002091B9063091BA064091BB065091BC06F5
:1025C0006091BD067091BE068091BF069091C006D5
:1025D0005101CB2EDA2EEF2EFE2E0EA11AA50E944F
:1025E000FA3589F01092B9061092BA061092BB061D
:1025F0001092BC061092BD061092BE061092BF0645
:102600001092C006A5CE4090A1061091A2061AA372
:102610008091A3068BA39091A4069CA30091A5068C
:102620000DA35090A6066090A7067090A806CE0154
:102630000D964C01A42CB12ECBA0DCA0E02EF52CE5
:10264000830191014B2F5A2F6F2F7E2F8EA19AA5B8
:102650000E94F30061E070E082E090E00E94F408E4
:1026600019A2298D3A8D4B8D5C8D6D8D7E8D8F8D50
:1026700098A130584A415640610971098109910970
:102680002F37304E42475849624071058105910508
:1026900009F008F4A3C082E08093C9062091B10636
:1026A0003091B2064091B3065091B4066091B506E0
:1026B0007091B6068091B7069091B806A0E00E948E
:1026C0000336F1F181EB96E00E94F7028FA3A09010
:1026D000A106B090A206C090A306D090A406E090F8
:1026E000A506F090A6060091A7061091A8062091D5
:1026F000B1063091B2064091B3065091B406609194
:10270000B5067091B606CE0101964C018091B706D0
:102710009091B8060E94F3001F928FA0A12CC9804F
:10272000DA80EB80FC800D811E812F813885498500
:102730005A856B857C8581E090E00E941A0F0F908E
:10274000898D8093B9068A8D8093BA068B8D80938C
:10275000BB068C8D8093BC068D8D8093BD068E8DBF
:102760008093BE068F8D8093BF0688A18093C0069C
:10277000BECE2093A1063093A2064093A3065093A9
:10278000A4066093A5067093A6068093A70690936F
:10279000A8068E01035F1F4F4801A12CB12CC12C4C
:1027A000D12CE12CF12C00E010E091014B2F5A2F9D
:1027B0006F2F7E2F8EA19AA50E94F300422E3AA37E
:1027C0004BA35CA36DA3572E3C0161E070E082E057
:1027D00090E00E94F40811E019A343CF88E08093B1
:1027E000C906AECFCF93DF93EC0188819981009722
:1027F00011F00E94C536198218821D821C821B822C
:102800001A82DF91CF910895FC01808191810C940F
:10281000C5360F931F93CF93DF938C01EB010E947A
:10282000A5328883C80101960E94A5328983CE0112
:10283000DF91CF911F910F910895CF92DF92EF9288
:10284000FF920F931F93CF93DF93EB017B0124E063
:10285000E20EF11C8B016C01C61AD70AC601800F6B
:10286000911F0E94A532F80181938F01EE15FF059B
:10287000A9F7CE01DF91CF911F910F91FF90EF90BB
:10288000DF90CF900895CF93DF93EB010E94A532A4
:102890008883CE01DF91CF9108950F931F93CF933B
:1028A000DF93EC0188819981009759F02A813B815F
:1028B0002617370730F081E0DF91CF911F910F91FC
:1028C00008958B016F5F7F4F0E944E37009759F03C
:1028D000998388831B830A832C813D81232B59F79D
:1028E000FC011082E8CF80E0E7CFEF92FF920F93D8
:1028F0001F93CF93DF936115710541F480E0DF9161
:10290000CF911F910F91FF90EF90089541155105C0
:10291000B1F07B01EC010C811D81040F151FB80182
:102920000E944D14882351F3288139818C819D8127
:10293000B701820F931F0E941D381D830C8381E015
:10294000DECFFC0101900020E9F73197AF01481B71
:10295000590BBC0189E696E00C947514EF92FF9236
:102960000F931F93CF93DF93EC017B018A01BA0190
:102970000E944D1481110BC0CE010E94F213CE01B2
:10298000DF91CF911F910F91FF90EF9008951D83DC
:102990000C83B701888199810E941D38F0CFFB011B
:1029A00001900020E9F73197AF01461B570B0C94BB
:1029B000AE14CF93DF93EC01FB018617970749F024
:1029C000608171816115710541F0448155810E94DA
:1029D000AE14CE01DF91CF9108950E94F213F9CF8A
:1029E000FC01118210821382128215821482FB0173
:1029F00001900020E9F73197AF01461B570B0C946B
:102A0000AE14FF920F931F93CF93DF93EC01F62E3A
:102A100008811981C8010E94A532F81621F06F2D96
:102A2000C8010E94AD32CE01DF91CF911F910F916D
:102A3000FF900895EF92FF920F931F93CF93DF9330
:102A400000D0CDB7DEB783E8E82E81E0F82E0FE1A5
:102A500010E01A830983F70161917F01CE0101968D
:102A60000E9401150F5F1F4F0332110591F783E894
:102A700091E00F900F90DF91CF911F910F91FF90F8
:102A8000EF900895EF92FF920F931F93CF93DF93F0
:102A900000D0CDB7DEB781E8E82E86E0F82E0EE252
:102AA00010E01A830983F70161917F01CE0101963D
:102AB0000E9401150F5F1F4F0433110591F781E844
:102AC00096E00F900F90DF91CF911F910F91FF90A3
:102AD000EF900895AF92BF92CF92DF92EF92FF9264
:102AE0000F931F93CF93DF9300D0CDB7DEB78B0149
:102AF0006B0124E0C20ED11C7B015C01A61AB70A4F
:102B0000C5018E0D9F1D9A838983F70161917F0115
:102B1000CE0101960E940115EC14FD0489F7C8014D
:102B20000F900F90DF91CF911F910F91FF90EF9039
:102B3000DF90CF90BF90AF900895EF92FF920F93E8
:102B40001F93CF93DF9300D0CDB7DEB78C017B010D
:102B50009A838983FB016081CE0101960E94011551
:102B60000F5F1F4F1A830983F7016181CE01019620
:102B70000E940115C7010F900F90DF91CF911F9117
:102B80000F91FF90EF9008950F931F930E94A90655
:102B90000091FF041091000520910105309102057C
:102BA000601B710B820B930B653F71408105910592
:102BB00008F4DEC161E080E00E944B0A82E192E00D
:102BC0000E94930B60918504709186048091870424
:102BD0009091880442E00E94920C83E892E00E9467
:102BE000930B8091DE048130C1F40E94A80760E05D
:102BF00080E00E944B0A8EE192E00E94930B80914C
:102C0000FD049091FE04909307018093060166E015
:102C100071E084E690E00E949D158091DE04823090
:102C2000D1F50E94A80760E080E00E944B0A80E393
:102C300092E00E94930B8091FD049091FE0490938A
:102C40004301809342012091060130910701821BCC
:102C5000930B63E070E00E943434260F371F3093EB
:102C6000050120930401260F371F30934101209363
:102C7000400164E071E087E690E00E949D1560E409
:102C800071E08AE690E00E949D1562E471E08DE6B5
:102C900090E00E949D158091DE048330D1F50E9462
:102CA000A80760E080E00E944B0A81E492E00E9465
:102CB000930B8091FD049091FE04909349018093C1
:102CC00048012091420130914301821B930B63E044
:102CD00070E00E943434260F371F30934501209353
:102CE0004401260F371F309347012093460164E4C7
:102CF00071E080E790E00E949D1566E471E083E753
:102D000090E00E949D1568E471E086E790E00E94E3
:102D10009D158091DE048430D1F50E94A80760E003
:102D200080E00E944B0A82E592E00E94930B809122
:102D3000FD049091FE0490934F0180934E012091E9
:102D4000480130914901821B930B63E070E00E94BF
:102D50003434260F371F30934B0120934A01260F3E
:102D6000371F30934D0120934C016AE471E089E7ED
:102D700090E00E949D156CE471E08CE790E00E9469
:102D80009D156EE471E08FE790E00E949D158091A3
:102D9000DE04853009F048C00E94A80760E080E0AA
:102DA0000E944B0A83E692E00E94930B8091FD04FF
:102DB0009091FE04909357018093560120914E010B
:102DC00030914F01821B930B97FD03969595879544
:102DD00095958795280F391F309351012093500105
:102DE000280F391F3093530120935201820F931FF4
:102DF000909355018093540160E571E082E890E082
:102E00000E949D1562E571E085E890E00E949D15A5
:102E100064E571E088E890E00E949D1566E571E048
:102E20008BE890E00E949D158091DE04863009F0C9
:102E300048C00E94A80760E080E00E944B0A84E737
:102E400092E00E94930B8091FD049091FE04909378
:102E50005F0180935E012091560130915701821BE2
:102E6000930B97FD03969595879595958795280FD4
:102E7000391F3093590120935801280F391F30937F
:102E80005B0120935A01820F931F90935D01809301
:102E90005C0168E571E08EE890E00E949D156AE5AE
:102EA00071E081E990E00E949D156CE571E084E994
:102EB00090E00E949D156EE571E087E990E00E9428
:102EC0009D158091DE04873009F048C00E94A80754
:102ED00060E080E00E944B0A85E892E00E94930B3C
:102EE0008091FD049091FE049093670180936601A8
:102EF00020915E0130915F01821B930B97FD039639
:102F00009595879595958795280F391F3093610181
:102F100020936001280F391F3093630120936201D1
:102F2000820F931F909365018093640160E671E0C6
:102F30008AE990E00E949D1562E671E08DE990E0DB
:102F40000E949D1564E671E080EA90E00E949D1564
:102F500066E671E083EA90E00E949D150E94A90652
:102F60006093FF0470930005809301059093020520
:102F70001F910F9108950F931F93CF93DF9300D06C
:102F8000CDB7DEB78B019A838983FB016081CE01C7
:102F900001960E940115C8010F900F90DF91CF910B
:102FA0001F910F910895CF9360E874E088E090E05E
:102FB0000E944314FC018081809380048091270546
:102FC000811112C066E972E081E896E00E94CF1498
:102FD0001092800460E874E088E090E00E94BB17E3
:102FE00060E080E10E94A405C0912705C13091F402
:102FF00061E674E081E896E00E94CF14C0938004FB
:1030000060E874E088E090E00E94BB1761E080E136
:103010000E94A40580912705823080F01092270538
:1030200066E972E081E896E00E94CF141092800475
:1030300060E874E088E090E00E94BB1767E275E00A
:1030400085E390E00E94BB17CF910C9442158F92BC
:103050009F92AF92BF92FF920F931F93CF93DF93F4
:10306000EC01F090290500912F0510913005F11029
:1030700052C00230110509F44EC08130910509F0AB
:10308000B6C08091DE048F5F873008F0AEC08093B9
:10309000DE0440916C0150916D0160916E01709160
:1030A0006F018091830190918401A0918501B0917D
:1030B0008601840F951FA61FB71F809383019093ED
:1030C0008401A0938501B093860160918301709182
:1030D0008401809185019091860120916C0130914D
:1030E0006D0140916E0150916F0180906C01909044
:1030F0006D01A0906E01B0906F010E944834C5012F
:10310000B4010E94243460938301709384018093FE
:103110008501909386018091830190918401A09113
:103120008501B0918601813C924CAA4DB64060F079
:1031300080EC92ECAAEDB6E0809383019093840139
:10314000A0938501B09386018091830190918401C1
:10315000A0918501B0918601803A9648A140B105C1
:1031600060F480EA96E8A1E0B0E080938301909358
:103170008401A0938501B093860121E0F212BBC0C7
:10318000C130D10509F082C040916C0150916D01B0
:1031900060916E0170916F018091EF049091F00445
:1031A000A091F104B091F204840F951FA61FB71FE0
:1031B0008093EF049093F004A093F104B093F20491
:1031C0000130110509F0D3C080912B0590912C0599
:1031D000A0912D05B0912E058093830190938401D9
:1031E000A0938501B09386019DC087E050CF0196E2
:1031F00009F091CF40916C0150916D0160916E0189
:1032000070916F018091830190918401A09185015B
:10321000B0918601841B950BA60BB70B809383019D
:1032200090938401A0938501B093860160918301FE
:1032300070918401809185019091860120916C01AB
:1032400030916D0140916E0150916F0180906C0141
:1032500090906D01A0906E01B0906F010E94483473
:10326000C501B4010E9424346093830170938401EA
:1032700080938501909386018091DE048150823095
:1032800018F08093DE0447CF81E0FBCFCF3FDC070F
:1032900009F0A4C240916C0150916D0160916E01E2
:1032A00070916F018091EF049091F004A091F1046E
:1032B000B091F204841B950BA60BB70B8093EF041F
:1032C0009093F004A093F104B093F204013011053F
:1032D00009F04DC080912B0590912C05A0912D05F2
:1032E000B0912E058093830190938401A093850172
:1032F000B09386018BC201301105C9F580912B0571
:1033000090912C05A0912D05B0912E0580938301FD
:1033100090938401A0938501B0938601C130D105BB
:1033200009F070C268E671E08AE190E00E941D1425
:1033300040916C0150916D0160916E0170916F012F
:10334000FC0180819181A281B381840F951FA61F0A
:10335000B71F8093680190936901A0936A01B093AD
:103360006B0168E671E08AE190E00E946A15809145
:103370002F05909130050297C9F5C130D10509F0AC
:1033800040C180912B0590912C05A0912D05B09105
:103390002E058093830190938401A0938501B093BF
:1033A00086016AE075E085E190E00E941D1440917D
:1033B0006C0150916D0160916E0170916F01FC0183
:1033C00080819181A281B381840F951FA61FB71FB1
:1033D00080937E0190937F01A0938001B09381013F
:1033E0006EE771E085E190E00E946A1580912F05FB
:1033F00090913005039759F580912B0590912C05FC
:10340000A0912D05B0912E058093830190938401A6
:10341000A0938501B0938601C130D10509F02BC17D
:103420008093830190938401A0938501B0938601DA
:103430006AE972E081E596E00E94CF1481E0809312
:10344000820162E871E08DE090E00E94BB178091FC
:103450002F0590913005049759F580912B05909197
:103460002C05A0912D05B0912E058093830190939A
:103470008401A0938501B0938601C130D10509F084
:103480000FC18093830190938401A0938501B09331
:1034900086016AE972E087E596E00E94CF1481E038
:1034A0008093260566E275E090E080E00E94BB17FD
:1034B00080912F05909130050597C9F5C130D10550
:1034C00009F003C180912B0590912C05A0912D0549
:1034D000B0912E058093830190938401A093850180
:1034E000B093860166E771E088E290E00E941D14C7
:1034F00040916C0150916D0160916E0170916F016E
:10350000FC0180819181A281B381840F951FA61F48
:10351000B71F8093760190937701A0937801B093C1
:10352000790166E771E088E290E00E946A15809177
:103530002F05909130050697C9F5C130D10509F0E6
:10354000FEC080912B0590912C05A0912D05B09186
:103550002E058093830190938401A0938501B093FD
:10356000860163E075E084E290E00E941D144091C2
:103570006C0150916D0160916E0170916F01FC01C1
:1035800080819181A281B381840F951FA61FB71FEF
:103590008093030590930405A0930505B093060559
:1035A00063E075E084E290E00E946A1580912F0547
:1035B000909130058730910509F003C1CF3FDC07BA
:1035C00009F0E9C080912B0590912C05A0912D0563
:1035D000B0912E058093830190938401A09385017F
:1035E000B09386016EE972E08BE496E0DF91CF91B3
:1035F0001F910F91FF90BF90AF909F908F900C9470
:10360000CF14CF3FDC0709F0F1CE80912B059091CC
:103610002C05A0912D05B0912E05809383019093E8
:103620008401A0938501B09386016AE075E085E18D
:1036300090E00E941D1440916C0150916D016091C9
:103640006E0170916F01FC0180819181A281B38133
:10365000841B950BA60BB70B181619061A061B062A
:103660000CF4B6CE10927E0110927F011092800170
:1036700010928101B5CECF3FDC0709F019CF8093BE
:10368000830190938401A0938501B09386016EE934
:1036900072E081E596E00E94CF1410928201D1CEB3
:1036A000CF3FDC0709F043CF8093830190938401DF
:1036B000A0938501B09386016EE972E087E596E0FC
:1036C0000E94CF1410922605EDCECF3FDC0709F003
:1036D0002ECF80912B0590912C05A0912D05B091B6
:1036E0002E058093830190938401A0938501B0936C
:1036F000860166E771E088E290E00E941D14409127
:103700006C0150916D0160916E0170916F01FC012F
:1037100080819181A281B381841B950BA60BB70B8D
:10372000181619061A061B060CF4F3CE1092760131
:10373000109277011092780110927901F2CECF3F6A
:10374000DC0709F033CF80912B0590912C05A091D7
:103750002D05B0912E058093830190938401A09351
:103760008501B093860163E075E084E290E00E94F9
:103770001D1440916C0150916D0160916E0170912A
:103780006F01FC0180819181A281B381841B950B23
:10379000A60BB70BFDCE219709F050C080912B05E9
:1037A00090912C05A0912D05B0912E058093830159
:1037B00090938401A0938501B09386016AE972E039
:1037C00013CF0897D9F5DF91CF911F910F91FF90FB
:1037D000BF90AF909F908F900C94C415013011054D
:1037E00009F0C5CD80912B0590912C05A0912D0558
:1037F000B0912E058093830190938401A09385015D
:10380000B0938601CF3FDC0709F0B1CD68E671E0E7
:103810008AE190E00E941D1440916C0150916D016D
:1038200060916E0170916F01FC0180819181A28194
:10383000B381841B950BA60BB70B8BCDDF91CF917A
:103840001F910F91FF90BF90AF909F908F90089520
:103850001F920F920FB60F9211242F933F934F9305
:103860005F936F937F938F939F93AF93BF93EF93E8
:10387000FF9382EA95E00E94C304FF91EF91BF910C
:10388000AF919F918F917F916F915F914F913F91F8
:103890002F910F900FBE0F901F9018951F920F92AF
:1038A0000FB60F9211242F938F939F93EF93FF9353
:1038B000E091B205F091B3058081E091B805F091F7
:1038C000B90582FD1BC090818091BB058F5F8F730E
:1038D0002091BC05821741F0E091BB05F0E0EE5568
:1038E000FA4F958F8093BB05FF91EF919F918F9138
:1038F0002F910F900FBE0F901F9018958081F4CFDD
:103900001F920F920FB60F9211242F933F938F9314
:103910009F93AF93BF938091CD049091CE04A091DB
:10392000CF04B091D0043091CC0423E0230F2D3785
:1039300058F50196A11DB11D2093CC048093CD04B0
:103940009093CE04A093CF04B093D0048091D1047F
:103950009091D204A091D304B091D4040196A11DFA
:10396000B11D8093D1049093D204A093D304B0935B
:10397000D404BF91AF919F918F913F912F910F9060
:103980000FBE0F901F90189526E8230F0296A11DD9
:10399000B11DD2CF1F920F920FB60F9211242F9309
:1039A0003F934F935F936F937F938F939F93AF93C7
:1039B000BF93EF93FF938091B900887F803609F41D
:1039C0004AC0F0F5883209F4A7C018F5803109F42F
:1039D0009BC0B8F4882309F4F9C0883009F494C076
:1039E000FF91EF91BF91AF919F918F917F916F91D7
:1039F0005F914F913F912F910F900FBE0F901F90AD
:103A00001895883109F488C0803251F780937B057E
:103A100014C0803409F49DC040F48033B9F3883376
:103A2000F9F680937B0585ECB0C0803509F485C03C
:103A3000883509F496C0883499F60E94B506D0CF2F
:103A4000883909F48CC038F5883729F050F4883665
:103A500011F0803729F683E080937D051092CB0426
:103A600057C0883809F47BC0803919F0803809F0D4
:103A7000B7CF8091CB04803208F071C0E091CB04C5
:103A800081E08E0F8093CB048091BB00F0E0E55580
:103A9000FB4F80833DC0803B39F0E0F4803A09F46D
:103AA00079C0883A09F09CCF84E080937D0510921C
:103AB000AA041092A904E0913305F0913405099508
:103AC0008091A90481110FC081E08093A904109214
:103AD000890409C0803C09F4A6CF883C09F4A3CF2F
:103AE000883B09F07DCFE091AA0481E08E0F80939E
:103AF000AA04F0E0E757FB4F80818093BB009091D0
:103B0000AA048091A90429C0809158058093BB0024
:103B100085EC8093BC0064CF90917A058091790503
:103B2000981758F5E0917A0581E08E0F80937A0519
:103B3000F0E0E75AFA4F8081E9CFE0917A0581E021
:103B40008E0F80937A058091BB00F0E0E75AFA4F20
:103B5000808390917A05809179059817C8F285E85D
:103B6000D8CFE0917A0581E08E0F80937A0580911D
:103B7000BB00F0E0E75AFA4F808380917C05811109
:103B80005CCF81E08093570584EA8093BC0010925B
:103B90007D0526CF85EC8093BC0010927D05809139
:103BA000CB04803230F4E091CB04F0E0E555FB4FDC
:103BB00010826091CB0470E0E0913105F091320504
:103BC0008BEA94E009951092CB040ACF10927B0502
:103BD00034CF1F920F920FB60F921124CF92DF9223
:103BE000EF92FF920F931F932F933F934F935F9307
:103BF0006F937F938F939F93AF93BF93CF93DF93F5
:103C0000EF93FF9380918F060E947B05EC018091DA
:103C10008E060E947B0590918D069F70CC0FDD1F54
:103C2000C82B24E0929FC001112483579E4FC80FD8
:103C3000D92FD11DC881C0938D06C07361F10E9438
:103C4000A9060091D5041091D6042091D704309193
:103C5000D8046B017C01C01AD10AE20AF30A970169
:103C600086010093DA041093DB042093DC04309384
:103C7000DD046093D5047093D6048093D7049093A9
:103C8000D80481E090E0C03121F0C03221F48FEF00
:103C90009FEF0E942718FF91EF91DF91CF91BF9185
:103CA000AF919F918F917F916F915F914F913F91D4
:103CB0002F911F910F91FF90EF90DF90CF900F9079
:103CC0000FBE0F901F901895CF93DF93E2EAF5E0B7
:103CD0001382128288EE93E0A0E0B0E084839583A3
:103CE000A683B7832DEA31E03183208325EC30E0D1
:103CF0003587248724EC30E03787268720EC30E0B6
:103D0000318B208B21EC30E0338B228B22EC30E0A6
:103D1000358B248B26EC30E0378B268B118E128E60
:103D2000138E148EEFE3F6E0138212828483958360
:103D3000A683B7838FEB91E091838083EEECF6E06E
:103D40001382128281ED91E09183808389E08483E4
:103D50008FEF8583C8E0C68387E0878386E080870E
:103D600085E0818784E0828713861486158616860F
:103D7000178681E00E94A509E0E9F6E0C0AFC1AF77
:103D800011AA12AA13AA1186128613861486158602
:103D900016861786108A118A128A138A148A158A3F
:103DA000168A178A108E118E128E138E148E158E0F
:103DB000168E178E10A211A212A213A214A215A27F
:103DC00016A217A210A611A612A613A614A615A62F
:103DD00016A617A610AA80E498E7ADE7B1E082AF77
:103DE00093AFA4AFB5AFCDE8D6E083E0898382E09E
:103DF0008A8360E083E00E94040660E08A810E947A
:103E0000040661E089810E94A40561E08A810E9424
:103E1000A405188262EA72E087E896E00E94F01436
:103E200066E972E081E896E00E94F01466E972E0CB
:103E30008BE796E00E94F01464EA72E085E796E072
:103E40000E94F01461E773E08FE696E00E94F014A0
:103E500061E773E089E696E00E94F01461E773E0A1
:103E600083E696E00E94F01461E773E08DE596E04A
:103E70000E94F0146EE972E087E596E00E94F0146B
:103E80006AE972E081E596E00E94F0146EE972E062
:103E90008BE496E0DF91CF910C94F014CF93DF93F5
:103EA000CDB7DEB7AF970FB6F894DEBF0FBECDBF6C
:103EB000789484B5826084BD84B5816084BD85B505
:103EC000826085BD85B5816085BD80916E00816011
:103ED00080936E00109281008091810082608093B7
:103EE00081008091810081608093810080918000B9
:103EF0008160809380008091B10084608093B100E4
:103F00008091B00081608093B00080917A008460DD
:103F100080937A0080917A00826080937A00809109
:103F20007A00816080937A0080917A008068809323
:103F30007A001092C100E091B205F091B30582E0E1
:103F40008083E091AE05F091AF051082E091B0055D
:103F5000F091B1058FEC80831092BA05E091B6051F
:103F6000F091B70586E08083E091B405F091B50546
:103F7000808180618083E091B405F091B5058081F6
:103F800088608083E091B405F091B50580818068F8
:103F90008083E091B405F091B50580818F7D8083A9
:103FA00082E00E94A50981E00E949F098BE39FE1C6
:103FB0000197F1F70E94D20561E08AE00E940406B1
:103FC00061E08BE00E94040661E08CE00E94040640
:103FD00061E08DE00E94040660E08FE00E9404062C
:103FE00061E080E10E94040661E081E10E94040634
:103FF00068E371E081E00E94600A60E371E082E0C2
:104000000E94600A68E271E083E00E94600A60E258
:1040100071E084E00E94600A68E171E085E00E943E
:10402000600A60E171E086E00E94600A68E071E089
:1040300087E00E94600A69ED74E089E090E00E94E8
:104040004314DC018C91813F09F4FBC666E275E004
:1040500090E080E00E94BB1781EF90E09A83898313
:10406000BE016F5F7F4F89E090E00E949D1562E87E
:1040700071E08DE090E00E94BB1762E175E08FE097
:1040800090E00E946A156EE771E085E190E00E9481
:104090006A1568E671E08AE190E00E946A150E9464
:1040A0001A1562E771E084E290E00E946A1566E703
:1040B00071E088E290E00E946A150E94421567E272
:1040C00075E085E390E00E94BB1760E771E087E34D
:1040D00090E00E949D1566E071E084E690E00E9409
:1040E0009D1564E071E087E690E00E949D1560E414
:1040F00071E08AE690E00E949D1562E471E08DE631
:1041000090E00E949D1564E471E080E790E00E94D9
:104110009D1566E471E083E790E00E949D1568E4D8
:1041200071E086E790E00E949D156AE471E089E7FE
:1041300090E00E949D156CE471E08CE790E00E9495
:104140009D156EE471E08FE790E00E949D1560E59B
:1041500071E082E890E00E949D1562E571E085E8DB
:1041600090E00E949D1564E571E088E890E00E946F
:104170009D1566E571E08BE890E00E949D1568E56D
:1041800071E08EE890E00E949D156AE571E081E99A
:1041900090E00E949D156CE571E084E990E00E943A
:1041A0009D156EE571E087E990E00E949D1560E63F
:1041B00071E08AE990E00E949D1562E671E08DE968
:1041C00090E00E949D1564E671E080EA90E00E9414
:1041D0009D1566E671E083EA90E00E949D1566E217
:1041E00075E090E080E00E944314DC018C918093A4
:1041F000260562E871E08DE090E00E944314FC0126
:104200008081809382016AE075E085E190E00E9400
:104210001D14FC0180819181A281B38180937E0174
:1042200090937F01A0938001B093810168E671E0D3
:104230008AE190E00E941D14FC0180819181A2819D
:10424000B3818093680190936901A0936A01B09350
:104250006B018FE190E00E94A5328093000180E223
:1042600090E00E94A5328093010181E290E00E94DB
:10427000A5328093020182E290E00E94A5328093F1
:1042800003018091000190910101A0910201B09180
:1042900003018093830190938401A0938501B093DF
:1042A000860163E075E084E290E00E941D14FC0149
:1042B00080819181A281B381809372019093730177
:1042C000A0937401B093750166E771E088E290E015
:1042D0000E941D14FC0180819181A281B381809391
:1042E000760190937701A0937801B093790191E8DA
:1042F000E92E96E0F92E0EE210E0C8010E94A532E8
:10430000D7018D937D010F5F1F4F04331105A9F76E
:1043100061E876E0CB010E94D91467E275E085E39D
:1043200090E00E944314FC0180818093270560E7A0
:1043300071E087E390E00E940914DC018D919C916B
:10434000909371018093700180916801909169014F
:10435000A0916A01B0916B018093C4069093C50649
:10436000A093C606B093C7060E94D20562E987EB08
:104370000E9465078FE00E94690840EC5CEF6BE9E2
:1043800071E04093CA065093CB066093CC067093BD
:10439000CD06682F6F738FE00E94650760E880E1AB
:1043A0000E94650760E881E10E94650760E882E19C
:1043B0000E9465076CE080E10E9465076CE081E186
:1043C0000E9465076CE082E10E94650760E281EB74
:1043D0000E94650760E881EB0E94650710E000E03D
:1043E00020E03EE249E556E761E170E080E090E0E0
:1043F0000E946A0D61E081E090E00E94DC0890E09C
:1044000080E00E94D00881E090E00E94D00882E025
:1044100090E00E94D00862EA72E087E896E00E948D
:10442000CF1462E08EE00E940406809168008460F0
:104430008093680080916D008C6080936D0078940B
:104440000E94A9066093D5047093D6048093D70484
:104450009093D80488EE93E0A0E0B0E08093DA0473
:104460009093DB04A093DC04B093DD040E94000B66
:104470008091070590910805019709F097C08091F8
:10448000DA049091DB04A091DC04B091DD04853660
:104490009105A105B105C0F00AE010E020E030E090
:1044A00000936C0110936D0120936E0130936F01A6
:1044B0002EE630E040E050E02093DA043093DB0455
:1044C0004093DC045093DD048091DA049091DB0486
:1044D000A091DC04B091DD048997A109B109CC97C2
:1044E000A105B105C0F482E390E0A0E0B0E08093C4
:1044F0006C0190936D01A0936E01B0936F0106E47F
:1045000010E020E030E00093DA041093DB04209305
:10451000DC043093DD048091DA049091DB04A091F7
:10452000DC04B091DD044F97A109B1090A97A105F8
:10453000B105C0F424E630E040E050E020936C0187
:1045400030936D0140936E0150936F0183E290E0D0
:10455000A0E0B0E08093DA049093DB04A093DC0445
:10456000B093DD048091DA049091DB04A091DC0427
:10457000B091DD044F97A105B105C0F408EE13E03A
:1045800020E030E000936C0110936D0120936E01E8
:1045900030936F012FE030E040E050E02093DA04E8
:1045A0003093DB044093DC045093DD0480912F05AD
:1045B00090913005892B11F40E94000B8EE00E942F
:1045C00040068EE00E9440067C019093E2048093B6
:1045D000E1046AE070E080E090E00E9477068EE0FF
:1045E0000E9440068EE00E944006092E000CAA0B95
:1045F000BB0BA7010F2C000C660B770B4C015D0168
:1046000033E0831A9108A108B108481559056A05D5
:104610007B0564F00396A11DB11D84179507A607BD
:10462000B70724F0F092EE04E092ED04E090ED0480
:10463000F090EE0445E8E41643E0F4060CF410C4F0
:104640001092E0048091DF04811106C060E081E1F6
:104650000E94A40510922A0580912A0580931605D0
:104660008091830190918401A0918501B091860190
:1046700080349244AF40B10508F420C58091830195
:1046800090918401A0918501B0918601803C964C67
:10469000AD42B10508F012C515B81092E4041092AD
:1046A000E30480912F0590913005009781F04091AF
:1046B000830150918401609185017091860140933E
:1046C0002B0550932C0560932D0570932E0520919A
:1046D0002A05213099F5892B89F5E090E504F090C1
:1046E000E6042FEFE21AF20AF092E604E092E50403
:1046F00084E10E944006BC01990F880B990B0E942F
:1047000088314B015C0185E10E944006BC01990F94
:10471000880B990B0E9488312B013C01AC019B0155
:10472000C501B4010E941A3487FDF3C561E080E041
:104730000E944B0A88EA92E00E94930B81E09091DC
:104740002905913009F080E091E020912A0521119E
:1047500090E0892309F406C180912F0590913005DE
:10476000892B09F0FFC080917A0190917B01A09183
:104770007C01B0917D01803A46E8940741E0A407AE
:10478000B1050CF057C68091830190918401A091EE
:104790008501B0918601805A9648A140B109B09533
:1047A000A095909581959F4FAF4FBF4F8093EF0499
:1047B0009093F004A093F104B093F2048091ED047F
:1047C0009091EE0487599109C197D0F48091EB0440
:1047D0009091EC04843691059CF401969093EC043E
:1047E0008093EB04C29761F41092EF041092F004EE
:1047F0001092F1041092F2041092EC041092EB0467
:104800000E94950BC0908301D0908401E0908501B7
:10481000F09086018091EF049091F004A091F10452
:10482000B091F204C80ED91EEA1EFB1EC0927A0196
:10483000D0927B01E0927C01F0927D0161E084E006
:104840000E944B0A80E20E947C0AC701B60120E464
:1048500032E44FE050E00E946A3469017A01C0926C
:10486000E704D092E804E092E904F092EA041AE046
:10487000C116D104E104F1041CF480E20E947C0A18
:10488000C701B6010E94D60A8EE20E947C0A60919E
:104890007A0170917B0180917C0190917D0120E4EF
:1048A00032E44FE050E00E946A3428EE33E040E00A
:1048B00050E00E946A3469017A01C092E704D09204
:1048C000E804E092E904F092EA0424E6C216D10476
:1048D000E104F10464F480E30E947C0A3AE0C31628
:1048E000D104E104F1041CF480E30E947C0AC701B6
:1048F000B6010E94D60A8EE20E947C0A60917A017B
:1049000070917B0180917C0190917D0128EE33E0D4
:1049100040E050E00E946A346B017C01C092E704E1
:10492000D092E804E092E904F092EA0444E6C41666
:10493000D104E104F10464F480E30E947C0A5AE0AB
:10494000C516D104E104F1041CF480E30E947C0A42
:10495000C701B6010E94D60A80E20E947C0A80E26A
:104960000E947C0A80912A0590912905892B09F0E3
:10497000FCC080912F0590913005892B09F0F5C07E
:1049800061E773E089E696E00E94CF140E94A807D1
:104990000E94A9060E94A906C090FF04D0900005BD
:1049A000E0900105F09002056C197D098E099F09C0
:1049B000643671058105910540F48091FD04909164
:1049C000FE049093FC048093FB040E94A9066C19DA
:1049D0007D098E099F09643671058105910598F05E
:1049E0000E94A9066C197D098E099F09683C710512
:1049F0008105910540F48091FD049091FE0490930F
:104A0000FA048093F9040E94A9066C197D098E09A5
:104A10009F09683C71058105910598F00E94A906DF
:104A20006C197D098E099F096C32714081059105D1
:104A300040F48091FD049091FE049093F8048093DB
:104A4000F7040E94A9066C197D098E099F096C3232
:104A500071408105910598F00E94A9066C197D09A5
:104A60008E099F09603971408105910540F480915C
:104A7000FD049091FE049093F6048093F5040E9447
:104A8000A9066C197D098E099F096039714081055D
:104A9000910598F00E94A9066C197D098E099F095D
:104AA000653F71408105910540F48091FD0490912E
:104AB000FE049093F4048093F3040E94A9066C19F9
:104AC0007D098E099F09653F71408105910508F4B4
:104AD0004AC08091FB049091FC042091F90430912C
:104AE000FA04820F931F2091F7043091F804820F8B
:104AF000931F2091F5043091F604820F931F2091AB
:104B0000F3043091F404820F931F65E070E00E947B
:104B100034347B017093FE046093FD0466E671E01B
:104B200083EA90E00E940914DC018D919C91E816C3
:104B3000F9060CF498C489EC92E00E94A11461E09B
:104B400084E00E944B0A69E676E08EEC96E00E94D3
:104B500037040E94A9066093FF04709300058093B8
:104B60000105909302050E94950B80912F0590916D
:104B70003005181619060CF03AC1019701F560E0EE
:104B800080E00E944B0A87EE93E00E94930B0E9404
:104B9000950B61E084E00E944B0A8FE693E00E944F
:104BA000930B609168017091690180916A01909105
:104BB0006B010E94D60A8EE993E00E94930B8091CC
:104BC0002F0590913005029761F40E94F50B60E08B
:104BD00080E00E944B0A89EF93E00E94930B0E94B1
:104BE000950B80912F0590913005039759F50E9400
:104BF000F50B60E080E00E944B0A8AE094E00E949E
:104C0000930B80918201811106C06EE972E081E50B
:104C100096E00E94CF1480918201813031F46AE9DC
:104C200072E081E596E00E94CF1461E080E00E948E
:104C30004B0A61E576E08EEC96E00E94370480E254
:104C40000E947C0A80912F0590913005049771F5A0
:104C500060E080E00E944B0A8BE194E00E94930B9D
:104C600080912605811106C06EE972E087E596E025
:104C70000E94CF1480912605813031F46AE972E0F8
:104C800087E596E00E94CF1461E080E00E944B0A25
:104C90008EE693E00E94930B67E576E08EEC96E05B
:104CA0000E9437048DE294E00E94930B80912F05BF
:104CB00090913005059719F560E080E00E944B0A5D
:104CC0008BE394E00E94930B0E94950B61E084E0DB
:104CD0000E944B0A8FE693E00E94930B609176014D
:104CE0007091770180917801909179010E94D60AA4
:104CF0008CE494E00E94930B80E20E947C0A8091F5
:104D00002F0590913005069701F560E080E00E9444
:104D10004B0A84E594E00E94930B0E94950B61E09E
:104D200084E00E944B0A8FE693E00E94930B60910F
:104D300003057091040580910505909106050E9478
:104D4000D60A8CE494E00E94930B80912F059091F9
:104D500030050797F1F460E080E00E944B0A85E699
:104D600094E00E94930B8FE693E00E94930B61E026
:104D700080E00E944B0A82E993E00E94930B6BE46F
:104D800076E08EEC96E00E94370486E893E00E947D
:104D9000930B80912F0590913005089741F58091F4
:104DA0004F0690915006892B11F100914B061091FE
:104DB0004C066EE972E0C8010E941438892B21F478
:104DC0001092300510922F056AE972E0C8010E9426
:104DD0001438892B11F40E94C41580912F059091ED
:104DE0003005099724F01092300510922F0590910C
:104DF000280580912705981731F00E94D3178091DC
:104E0000270580932805809170019091710100978A
:104E100009F05EC421E030E03093080520930705D7
:104E200004EF11E020E030E08530910509F078C40E
:104E300000936C0110936D0120936E0130936F010C
:104E40007FC48EE00E944006853F91400CF4C7C9A4
:104E50008EE00E9440068A3892400CF4F7C8BFC921
:104E600058E4E516F1046CF48091E004811109C066
:104E700061E081E10E94A40581E080932A0580938E
:104E8000E004C701895491098D34910538F580916A
:104E9000E004811123C08091DF0481110BC061E027
:104EA00081E10E94A40581E08093DF0480932A05BC
:104EB0008093E0048091E0048111CECB1091DF0457
:104EC000113009F0C9CB60E081E10E94A405109285
:104ED000DF0410922A051093E004BECBC701875966
:104EE00091098034910508F58091E00481111DC07D
:104EF00080912905811109C081E080932905809363
:104F0000E0041092EC041092EB048091E004811113
:104F10000CC080912905813041F4109229058093BD
:104F2000E0041092EC041092EB04C701885D910933
:104F3000C697D8F48091E004811117C08091E304F2
:104F40009091E40401968A3091052CF49093E40446
:104F50008093E30404C01092E4041092E30481E01F
:104F60008093E0040E94CA0777CBC7018F5091401D
:104F7000C19770F48091E00481110AC08091E3042C
:104F80009091E404019797FFE1CF89E090E0DECFB4
:104F9000C701815491408C9708F58091E0048111FC
:104FA0001DC080910905811105C081E0809309052C
:104FB0008093E0048091E004811108C0809109058C
:104FC000813021F4109209058093E0048091270537
:104FD0008F5F809327050E94D3173ECBC7018E5663
:104FE00091408297D8F48091E004811117C080919C
:104FF0001D05811105C081E080931D058093E004AB
:105000008091E004811128CB80911D05813009F049
:1050100023CB10921D058093E0041ECBC70181595C
:1050200091408297B8F48091E004811113C080917F
:105030007001909171010196893091052CF4909343
:1050400071018093700104C010927101109270017F
:1050500081E0E1CFC7018F5A91408336910570F40A
:105060008091E00481110AC08091700190917101DA
:10507000019797FFE4CF88E090E0E1CF83E1E81A61
:1050800082E0F80A97E7E916F10408F0E5CA809192
:10509000E0048111E1CA80912F05909130050196BD
:1050A0009093300580932F0521E02093DE0409972B
:1050B0007CF21092300510922F05CACF80918301A7
:1050C00090918401A0918501B0918601803C964C1D
:1050D000AD42B10570F08091830190918401A0915F
:1050E0008501B091860180349B44AC44B10508F43D
:1050F00090C08091830190918401A0918501B0912D
:10510000860180349B44AC44B10508F08BC080918B
:10511000830190918401A0918501B0918601811550
:105120009241AA47B10570F080918301909184016A
:10513000A0918501B091860181159B41A74BB105D6
:1051400008F483C08091830190918401A09185012E
:10515000B091860181159B41A74BB10508F07AC03B
:105160008091830190918401A0918501B091860185
:1051700081159442A44FB10508F07FC0809183014E
:1051800090918401A0918501B0918601803C9A4E56
:10519000A142B14008F084C08091830190918401C4
:1051A000A0918501B09186018038914BAF44B14008
:1051B00008F089C08091830190918401A0918501BC
:1051C000B0918601803C9C4FAB49B14008F08EC045
:1051D0008091830190918401A0918501B091860115
:1051E00081159A45A246B24008F45BCA80918301BA
:1051F00090918401A0918501B0918601813C9B43EF
:10520000A744B34008F04DCA84E285B989E090E034
:1052100004C084E085B981E090E09093E404809339
:10522000E3043FCA8091830190918401A09185019C
:10523000B091860181159241AA47B10508F067CF68
:1052400088E085B982E090E0E8CF8CE085B983E022
:1052500090E0E3CF8091830190918401A09185013A
:10526000B091860181159442A44FB10508F078CF22
:1052700080E185B984E090E0D0CF80918301909166
:105280008401A0918501B0918601803C9A4EA14293
:10529000B14008F073CF84E185B985E090E0BDCFDF
:1052A0008091830190918401A0918501B091860144
:1052B0008038914BAF44B14008F06ECF88E185B99A
:1052C00086E090E0AACF8091830190918401A09123
:1052D0008501B0918601803C9C4FAB49B14008F0FC
:1052E00069CF8CE185B987E090E097CF8091830109
:1052F00090918401A0918501B091860181159A4514
:10530000A246B24008F064CF80E285B988E090E020
:1053100084CF34E1E316F1040CF410CA1092E604D1
:105320001092E504A3019201C501B4010E940D335E
:105330006B017C01A5019401C301B2010E940C33F1
:105340009B01AC01C701B6010E9479336B017C015E
:1053500020E030E0A9010E941A34181624F0F7FA70
:10536000F094F7F8F09420E030E040EA50E4C30114
:10537000B2010E94E73120E030EC4FE754E40E9494
:1053800079332CE238E540EB5CE30E9479339B01F2
:10539000AC010E94E73120E030E048E452E40E9492
:1053A00079334B015C0120E030E040E050E4C7017C
:1053B000B6010E940D332B013C01A701960160E06C
:1053C00070E080E89FE30E9479339B01AC01C30148
:1053D000B2010E940D339B01AC0160E070E080E8F7
:1053E00090E40E947933A50194010E94E7314B01BA
:1053F0005C0161E080E00E944B0A8BEB92E00E942E
:10540000930B42E0C701B6010E94920C61E088E074
:105410000E944B0A80EC92E00E94930B61E08BE0CB
:105420000E944B0A40E0C501B4010E94920C84EC3A
:1054300092E082C9813C924CAA4DB6400CF4BEC9A0
:105440008091830190918401A0918501B0918601A2
:1054500000EC12EC2AED36E0081B190B2A0B3B0B73
:10546000D901C801A3C966E671E083EA90E00E9411
:105470000914FC01808191818E159F051CF486ED35
:1054800092E05BCB64E671E080EA90E00E94091450
:10549000DC018D919C918E159F051CF483EE92E0AA
:1054A0004CCB62E671E08DE990E00E940914FC01AA
:1054B000808191818E159F051CF480EF92E03DCB99
:1054C00060E671E08AE990E00E940914DC018D91A8
:1054D0009C918E159F051CF48DEF92E02ECB6EE50E
:1054E00071E087E990E00E940914FC0180819181BC
:1054F0008E159F051CF48AE093E01FCB6CE571E0EC
:1055000084E990E00E940914DC018D919C918E1534
:105510009F051CF487E193E010CB6AE571E081E917
:1055200090E00E940914FC01808191818E159F05F5
:105530001CF484E293E001CB68E571E08EE890E032
:105540000E940914DC018D919C918E159F051CF41D
:1055500081E393E0F2CA66E571E08BE890E00E9497
:105560000914FC01808191818E159F051CF48EE346
:1055700093E0E3CA64E571E088E890E00E940914D2
:10558000DC018D919C918E159F051CF48BE493E0BA
:10559000D4CA62E571E085E890E00E940914FC013C
:1055A000808191818E159F051CF488E593E0C5CA22
:1055B00060E571E082E890E00E940914DC018D91C1
:1055C0009C918E159F051CF485E693E0B6CA6EE4A7
:1055D00071E08FE790E00E940914FC0180819181C5
:1055E0008E159F051CF482E793E0A7CA6CE471E076
:1055F0008CE790E00E940914DC018D919C918E153E
:105600009F051CF48FE793E098CA6AE471E089E78C
:1056100090E00E940914FC01808191818E159F0504
:105620001CF48CE893E089CA68E471E086E790E0B6
:105630000E940914DC018D919C918E159F051CF42C
:1056400089E993E07ACA66E471E083E790E00E941A
:105650000914FC01808191818E159F051CF486EA56
:1056600093E06BCA64E471E080E790E00E94091463
:10567000DC018D919C918E159F051CF483EB93E0CA
:105680005CCA62E471E08DE690E00E940914FC01BE
:10569000808191818E159F051CF480EC93E04DCAAA
:1056A00060E471E08AE690E00E940914DC018D91CB
:1056B0009C918E159F051CF48DEC93E03ECA60E42E
:1056C00071E087E690E00E9409148AED93E035CA04
:1056D0008130910589F441E050E060E070E0409352
:1056E0006C0150936D0160936E0170936F01109285
:1056F00008051092070594CB8230910509F0E8C0A7
:105700000AE010E020E030E000936C0110936D019E
:1057100020936E0130936F011092080510920705D7
:105720008630910509F0E7C028EE33E040E050E014
:1057300020936C0130936D0140936E0150936F0183
:10574000109208051092070560E771E087E390E08A
:105750000E949D158091120590911305A09114054A
:10576000B091150580930E0590930F05A093100539
:10577000B09311056AE075E085E190E00E941D1488
:10578000FC0180819181A281B38180937E019093FD
:105790007F01A0938001B093810190902A05F1E0F0
:1057A0009F1210C08091830190918401A091850186
:1057B000B091860180937A0190937B01A0937C0144
:1057C000B0937D018091830190918401A091850126
:1057D000B0918601A0901D05B0902905C0907A0176
:1057E000D0907B01E0907C01F0907D0180389F4952
:1057F000A54DB10508F44DC1A110D5C062EA72E013
:1058000087E896E00E94CF1464EA72E085E796E0AC
:105810000E94CF1411E0B1128FC0409176015091D7
:105820007701609178017091790140907E015090EC
:105830007F016090800170908101D701C601840FC3
:10584000951FA61FB71F00911205109113052091F7
:10585000140530911505800F911FA21FB31F88A753
:1058600099A7AAA7BBA7840D951DA61DB71D809358
:10587000220590932305A0932405B0932505440D9C
:10588000551D661D771D40937E0150937F016093E7
:1058900080017093810180910905813009F03FC139
:1058A00091E099123CC18091220590912305A0912D
:1058B0002405B091250540917201509173016091CA
:1058C000740170917501841B950BA60BB70BB9C0C1
:1058D00083309105C1F422E330E040E050E02093B2
:1058E0006C0130936D0140936E0150936F011092E3
:1058F00008051092070587309105B1F480E197E221
:10590000A0E0B0E008C08430910509F089CA84E6BF
:1059100090E0A0E0B0E080936C0190936D01A093C3
:105920006E01B0936F010CCF089709F00DCF00EA1C
:1059300016E821E030E07CCAB110ADCF20918301A0
:1059400030918401409185015091860128A739A7A3
:105950004AA75BA740917601509177016091780149
:105960007091790140907E0150907F01609080019C
:10597000709081018091120590911305A0911405FA
:10598000B09115058C019D01040F151F261F371FAF
:1059900088A599A5AAA5BBA5080F191F2A1F3B1FFB
:1059A000D901C80160CFA1E0AA1273C065E774E015
:1059B00087E896E00E94CF1467E774E085E796E0F9
:1059C0000E94CF14B1E0BB1245C0809112059091A6
:1059D0001305A0911405B09115058C0D9D1DAE1DEC
:1059E000BF1D40917E0150917F01609180017091B7
:1059F0008101840F951FA61FB71F809322059093E6
:105A00002305A0932405B0932505809109058130D5
:105A100009F085C0E1E09E1282C08091220590913C
:105A20002305A0912405B091250540917201509164
:105A300073016091740170917501840F951FA61F09
:105A4000B71F8093220590932305A0932405B0935C
:105A5000250565C0B110D9CF4091830150918401D3
:105A600060918501709186018091120590911305D6
:105A7000A0911405B091150540907E0150907F01D2
:105A80006090800170908101840D951DA61DB71D49
:105A9000B0CF8091830190918401A0918501B09154
:105AA000860180389F49A54DB105C8F5A110AFC04A
:105AB00065E774E087E896E00E94CF1464EA72E03C
:105AC00085E796E00E94CF1401E0B01281C080917A
:105AD000120590911305A0911405B09115058C0D38
:105AE0009D1DAE1DBF1D40917E0150917F016091B3
:105AF000800170918101840F951FA61FB71F8093AD
:105B0000220590932305A0932405B0932505809149
:105B10000905813021F411E0911609F47ECF960138
:105B2000A70126013701770C4408542C3201642D5B
:105B3000742D842D942D2F373F49454D5105610516
:105B400071058105910509F008F424C1A110D9C09F
:105B5000B1E0BB124BC18091120590911305A09149
:105B60001405B09115058C0D9D1DAE1DBF1D4091F6
:105B70007E0150917F016091800170918101840FBD
:105B8000951FA61FB71F8093220590932305A0930E
:105B90002405B093250580910905813009F026C1BF
:105BA000E1E09E1223C18091220590912305A091EE
:105BB0002405B091250540917201509173016091C7
:105BC000740170917501841B950BA60BB70BD9C09E
:105BD000B1109DCF40918301509184016091850166
:105BE000709186018091120590911305A091140582
:105BF000B091150540907E0150907F01609080012A
:105C000070908101840D951DA61DB71D74CF21E0F4
:105C1000A21285CF62EA72E087E896E00E94CF1474
:105C200067E774E085E796E00E94CF1431E0B31295
:105C300031C0409176015091770160917801709167
:105C4000790140907E0150907F01609080017090BA
:105C50008101D701C601840F951FA61FB71F8C01B4
:105C60009D01040D151D261D371D80911205909173
:105C70001305A0911405B0911505080F191F2A1FCF
:105C80003B1F009322051093230520932405309396
:105C90002505F5CDB110FFCD809183019091840150
:105CA000A0918501B09186014090760150907701D6
:105CB000609078017090790140917E0150917F0150
:105CC0006091800170918101440D551D661D771D05
:105CD000840F951FA61FB71F409012055090130503
:105CE0006090140570901505840D951DA61DB71DB7
:105CF0008093220590932305A0932405B093250556
:105D0000C2CDF1E0AF1272C0BF1270C08091120517
:105D100090911305A0911405B09115058C0D9D1D52
:105D2000AE1DBF1D40917E0150917F0160918001A9
:105D300070918101840F951FA61FB71F80932205C4
:105D400090932305A0932405B09325058091090520
:105D5000813009F04BC09F1249C08091220590917B
:105D60002305A0912405B091250540917201509121
:105D700073016091740170917501840F951FA61FC6
:105D8000B71F8093220590932305A0932405B09319
:105D900025052CC0A11086C001E0B01227C080915B
:105DA0007E0190917F01A0918001B09181018C0DC5
:105DB0009D1DAE1DBF1D40911205509113056091B0
:105DC000140570911505840F951FA61FB71F8093AA
:105DD000220590932305A0932405B0932505809177
:105DE0000905813019F4901609F4B7CF8091260582
:105DF000813029F461E081E090E00E94DC0880912C
:105E00002605811105C060E081E090E00E94DC0879
:105E100080918201811105C060E082E090E00E94E3
:105E2000DC0880918201813029F461E082E090E019
:105E30000E94DC08409122055091230560912405C1
:105E40007091250580911E0590911F05A091200558
:105E5000B0912105481759076A077B0709F0E8C088
:105E6000209185063091860680917F06909180066C
:105E70002817390709F0DCC08091810690918206CD
:105E800060917B0670917C06009709F4A7C06115AC
:105E9000710509F040C0232B09F4ADC0FC018081DD
:105EA00090E0A7C011E0A112A1CFB1129FCF8091C5
:105EB0007E0190917F01A0918001B09181018C0DB4
:105EC0009D1DAE1DBF1D409112055091130560919F
:105ED000140570911505840F951FA61FB71F4091DB
:105EE0007601509177016091780170917901840F6A
:105EF000951FA61FB71F8093220590932305A0939B
:105F00002405B093250580910905813009F06ECFF5
:105F100091126CCF48CE0E9414386BC00E94C536D7
:105F20008AA19BA190935E0680935D068CA19DA1A2
:105F30009093600680935F068EA19FA19093620666
:105F4000809361061BA21AA21DA21CA217C16BE7B7
:105F500074E0CE0101960E94F014409161065091C8
:105F6000620660915D0670915E06CE0101960E9408
:105F70007514811104C0CE0101960E94F21341E014
:105F800050E06EE774E0CE0101960E947514811115
:105F900004C0CE0101960E94F213BE016F5F7F4FD5
:105FA00082EA95E00E943704CE0101960E94041413
:105FB00064E170E080E090E00E94770680E090E08D
:105FC000892B11F40C9438220E94AF04882311F419
:105FD0000C9438220E9400000C943822611571053F
:105FE00051F0232B41F0DB018C9190E0919581954C
:105FF0009109892BE9F480911C058A1119C08091BF
:106000001B05B81215C040917E0150917F0160912F
:106010008001709181018091170590911805A091E0
:106020001905B0911A05481759076A077B0731F21D
:10603000609122057091230580912405909125059A
:1060400024E630E040E050E00E94F03410E000E050
:106050000E94D60F60918301709184018091850127
:106060009091860124E630E040E050E00E94F03458
:1060700001E010E00E94D60F60917E0170917F01D7
:10608000809180019091810124E630E040E050E071
:106090000E94E13402E010E00E94D60FB0921B058E
:1060A0008091220590912305A0912405B0912505AA
:1060B00080931E0590931F05A0932005B0932105A2
:1060C00061E876E08BE796E00E94D914A0921C0567
:1060D0008091160580932A0580917E0190917F0121
:1060E000A0918001B09181018093170590931805CC
:1060F000A0931905B0931A050E941A156AE070E082
:1061000080E090E00E9477066091830170918401A5
:1061100080918501909186011BA21AA21DA21CA24A
:106120001FA21EA22AE0AE014F5F5F4F0E943531D1
:10613000BE016F5F7F4FCE0182960E94CF14809187
:106140005D0690915E06009709F4EACE6AA17BA1F4
:106150006115710509F4E2CE40915F065091600629
:106160002EA13FA14217530708F4D8CE0E941D3834
:106170008EA19FA190936206809361061FA21EA22A
:10618000CE0182960E94041480916106909162066D
:106190000B9708F0DCCE1BA21AA21DA21CA21FA204
:1061A0001EA24AE0BE016F5F7F4F90E080E00E9438
:1061B0002A31BE016F5F7F4FCE0182960E94CF14BD
:1061C000409161065091620660915D0670915E0695
:1061D000CE0182960E947514811104C0CE01829670
:1061E0000E94F213BE016E5D7F4F8DE596E00E9426
:1061F000D914CE0182960E940414C6CF8BE496E097
:106200000E94041481E596E00E94041487E596E05C
:106210000E9404148DE596E00E94041483E696E043
:106220000E94041489E696E00E9404148FE696E02A
:106230000E94041485E796E00E9404148BE796E020
:106240000E94041481E896E00E94041487E896E016
:106250000C940414BB274A3031F4992322F4BDE294
:10626000909581959F4F0C945831BB27FA01A62F2A
:106270006217710581059105330B30FB66F0AA2783
:10628000660F771F881F991FAA1FA21710F0A21B65
:1062900063953850A9F7A05DAA3308F0A95DA193D2
:1062A00036F7B111B1931082CA010C947131BB273A
:1062B000FB015527AA27880F991FAA1FA41710F0C2
:1062C000A41B83955051B9F7A05DAA3308F0A95DCE
:1062D000A193009779F7B111B1931192CB010C946E
:1062E0007131DC01FC01672F71917723E1F732975F
:1062F00004C07C916D9370836291AE17BF07C8F3A1
:1063000008950E94C33108F481E00895E89409C01B
:1063100097FB3EF490958095709561957F4F8F4FD8
:106320009F4F9923A9F0F92F96E9BB279395F695EE
:10633000879577956795B795F111F8CFFAF4BB0F6C
:1063400011F460FF1BC06F5F7F4F8F4F9F4F16C0D0
:10635000882311F096E911C0772321F09EE8872F5A
:10636000762F05C0662371F096E8862F70E060E016
:106370002AF09A95660F771F881FDAF7880F96958F
:10638000879597F90895990F0008550FAA0BE0E833
:10639000FEEF16161706E807F907C0F012161306E7
:1063A000E407F50798F0621B730B840B950B39F427
:1063B0000A2661F0232B242B252B21F408950A268D
:1063C00009F4A140A6958FEF811D811D08950E94BB
:1063D000FA310C946B320E945D3238F00E946432C4
:1063E00020F0952311F00C9454320C945A3211245D
:1063F0000C949F320E947C3270F3959FC1F3950FED
:1064000050E0551F629FF001729FBB27F00DB11D38
:10641000639FAA27F00DB11DAA1F649F6627B00DC8
:10642000A11D661F829F2227B00DA11D621F739FB1
:10643000B00DA11D621F839FA00D611D221F749FBF
:106440003327A00D611D231F849F600D211D822F06
:10645000762F6A2F11249F5750409AF0F1F088232D
:106460004AF0EE0FFF1FBB1F661F771F881F91505A
:106470005040A9F79E3F510580F00C9454320C9483
:106480009F325F3FE4F3983ED4F386957795679506
:10649000B795F795E7959F5FC1F7FE2B880F911D84
:1064A0009695879597F9089597F99F6780E870E02A
:1064B00060E008959FEF80EC089500240A9416167A
:1064C000170618060906089500240A9412161306E2
:1064D000140605060895092E0394000C11F4882370
:1064E00052F0BB0F40F4BF2B11F460FF04C06F5F8C
:1064F0007F4F8F4F9F4F089557FD9058440F551F62
:1065000059F05F3F71F04795880F97FB991F61F035
:106510009F3F79F087950895121613061406551FAC
:10652000F2CF4695F1DF08C0161617061806991F18
:10653000F1CF86957105610508940895E894BB270D
:1065400066277727CB0197F90895F999FECF92BD79
:1065500081BDF89A992780B50895262FF999FECF25
:106560001FBA92BD81BD20BD0FB6F894FA9AF99A70
:106570000FBE019608950E94FD32A59F900DB49F15
:10658000900DA49F800D911D112408952F923F928C
:106590004F925F926F927F928F929F92AF92BF9233
:1065A000CF92DF92EF92FF920F931F93CF93DF93DF
:1065B000CDB7DEB7CA1BDB0B0FB6F894DEBF0FBE3C
:1065C000CDBF09942A88398848885F846E847D8489
:1065D0008C849B84AA84B984C884DF80EE80FD808B
:1065E0000C811B81AA81B981CE0FD11D0FB6F89401
:1065F000DEBF0FBECDBFED010895A29FB001B39FD6
:10660000C001A39F700D811D1124911DB29F700DBB
:10661000811D1124911D08955058BB27AA270E945F
:1066200024330C946B320E945D3238F00E94643245
:1066300020F039F49F3F19F426F40C945A320EF4EA
:10664000E095E7FB0C945432E92F0E947C3258F31A
:10665000BA17620773078407950720F079F4A6F547
:106660000C949E320EF4E0950B2EBA2FA02D0B0148
:10667000B90190010C01CA01A0011124FF27591B87
:1066800099F0593F50F4503E68F11A16F040A22F8D
:10669000232F342F4427585FF3CF469537952795FE
:1066A000A795F0405395C9F77EF41F16BA0B620BFD
:1066B000730B840BBAF09150A1F0FF0FBB1F661F44
:1066C000771F881FC2F70EC0BA0F621F731F841F87
:1066D00048F4879577956795B795F7959E3F08F0AD
:1066E000B0CF9395880F08F09927EE0F979587956F
:1066F00008950E948D330C946B320E94643258F0DE
:106700000E945D3240F029F45F3F29F00C9454322E
:1067100051110C949F320C945A320E947C3268F3CF
:106720009923B1F3552391F3951B550BBB27AA274A
:1067300062177307840738F09F5F5F4F220F331F84
:10674000441FAA1FA9F335D00E2E3AF0E0E832D04C
:1067500091505040E695001CCAF72BD0FE2F29D04F
:10676000660F771F881FBB1F261737074807AB0721
:10677000B0E809F0BB0B802DBF01FF2793585F4F96
:106780003AF09E3F510578F00C9454320C949F32AD
:106790005F3FE4F3983ED4F3869577956795B79578
:1067A000F7959F5FC9F7880F911D9695879597F983
:1067B0000895E1E0660F771F881FBB1F62177307FC
:1067C0008407BA0720F0621B730B840BBA0BEE1F11
:1067D00088F7E09508950E94843288F09F5798F0DA
:1067E000B92F9927B751B0F0E1F0660F771F881FD6
:1067F000991F1AF0BA95C9F714C0B13091F00E94F0
:106800009E32B1E008950C949E32672F782F88272E
:10681000B85F39F0B93FCCF3869577956795B39516
:10682000D9F73EF490958095709561957F4F8F4F85
:106830009F4F08950E94C33108F48FEF08950E947E
:10684000C331880B990B0895DB018F939F930E94AE
:10685000BB32BF91AF91A29F800D911DA39F900D60
:10686000B29F900D1124089597FB072E16F4009403
:1068700007D077FD09D00E940F3607FC05D03EF403
:10688000909581959F4F0895709561957F4F0895DC
:10689000A1E21A2EAA1BBB1BFD010DC0AA1FBB1F24
:1068A000EE1FFF1FA217B307E407F50720F0A21B96
:1068B000B30BE40BF50B661F771F881F991F1A9403
:1068C00069F760957095809590959B01AC01BD012D
:1068D000CF010895052E97FB1EF400940E94813489
:1068E00057FD07D00E94483407FC03D04EF40C94A7
:1068F000813450954095309521953F4F4F4F5F4FD4
:10690000089590958095709561957F4F8F4F9F4F1B
:106910000895DF93CF931F930F939A9DF02D219F9E
:10692000F00D8B9DF00D8A9DE02DF10D039FF00D74
:10693000029FE00DF11D4E9DE00DF11D5E9DF00DDD
:106940004F9DF00D7F936F93BF92AF925F934F93E4
:10695000D5010E94FD328B01AC01D7010E94FD32AE
:10696000EB01E80FF91FD6010E94D8342F913F9117
:10697000D6010E94FD32C60FD71FE81FF91FAF9145
:10698000BF910E94D8342F913F910E94FD32C60FD3
:10699000D71FE81FF91FD6010E94FD32E60FF71F2F
:1069A0009801BE01CF010F911F91CF91DF91089502
:1069B0000E94FD32460F571FC81FD91F08F4319699
:1069C000089597FB57FF0C94F1349F938F930E9487
:1069D000F1346E1B7F0BAF91BF918A0B9B0B089517
:1069E000E894DF93CF93FC01DB010E94FD327F939B
:1069F0006F93E9019A01AC01BF93AF933F932F933B
:106A0000DF010E94FD3226F46C1B7D0B820B930B81
:106A10009E01EB01FC010E94D834AF91BF912F91F0
:106A20003F910E94D834BE01CF01F9012F913F91CF
:106A3000CF91DF910895689401C0E894F92FF12B6C
:106A400012F00C944F35A0E0B0E0E9E2F5E30C94CD
:106A5000CC32092E059422F40E94AB35112392F416
:106A6000F0E80F26FFEFE094F09400951095B094B5
:106A7000C094D094A194BF0ACF0ADF0AEF0AFF0A9C
:106A80000F0B1F0B0E945A3507FC0E94AB35CDB788
:106A9000DEB7ECE00C94E832689401C0E8948F9281
:106AA0009F92CF93DF930E945A35DF91CF919F90B1
:106AB0008F90089588249924F401E401B0E49F9311
:106AC000AA279A158B049C04ED05FE05CF05D00777
:106AD000A10798F4AD2FDC2FCF2FFE2FE92D982C96
:106AE000892E982F872F762F652F542F432F322FE3
:106AF0002227B85031F7BF9127C01B2EBF91BB276B
:106B0000220F331F441F551F661F771F881F991FB1
:106B1000881C991CEE1FFF1FCC1FDD1FAA1FBB1F67
:106B20008A149B04EC05FD05CE05DF05A007B1071F
:106B300048F08A189B08EC09FD09CE09DF09A00B73
:106B4000B10B21601A94E1F62EF49401AF01BE015D
:106B5000CD01000C089560957095809590953095C5
:106B60004095509521953F4F4F4F5F4F6F4F7F4F4F
:106B70008F4F9F4F0895002E083090F0982F872F49
:106B8000762F652F542F432F322F22270850F4CF12
:106B9000220F331F441F551F661F771F881F991F21
:106BA0000A95B2F7002D089597FD1094002E083035
:106BB00098F00850232F342F452F562F672F782F0A
:106BC000892F912DF4CF1594979587957795679593
:106BD00057954795379527950A95AAF71124002DC3
:106BE00008952A0D3B1D4C1D5D1D6E1D7F1D801FD0
:106BF000911F08952A153B054C055D056E057F051F
:106C00008007910708950024A7FD00942A173005F6
:106C10004005500560057005800590050895AA1B84
:106C2000BB1B51E107C0AA1FBB1FA617B70710F077
:106C3000A61BB70B881F991F5A95A9F780959095A9
:106C4000BC01CD010895EE0FFF1F0590F491E02DDA
:106C500009940F931F93CF93DF938230910510F423
:106C600082E090E0E091E806F091E90630E020E073
:106C7000B0E0A0E0309799F42115310509F44AC03D
:106C8000281B390B24303105D8F58A819B81611589
:106C9000710589F1FB0193838283FE0111C040815C
:106CA00051810281138148175907E0F048175907AD
:106CB00099F4109761F012960C93129713961C9307
:106CC0003296CF01DF91CF911F910F9108950093DC
:106CD000E8061093E906F4CF2115310551F042176B
:106CE000530738F0A901DB019A01BD01DF01F8016A
:106CF000C1CFEF01F9CF9093E9068093E806CDCF9D
:106D0000FE01E20FF31F81939193225031093983E1
:106D10002883D7CF2091E6063091E706232B41F454
:106D20002091890130918A013093E7062093E6068D
:106D300020918701309188012115310541F42DB74B
:106D40003EB740918B0150918C01241B350BE09193
:106D5000E606F091E706E217F307A0F42E1B3F0BBF
:106D60002817390778F0AC014E5F5F4F24173507BD
:106D700048F04E0F5F1F5093E7064093E60681935D
:106D800091939FCFF0E0E0E09CCFCF93DF9300970B
:106D9000E9F0FC01329713821282A091E806B091CB
:106DA000E906ED0130E020E01097A1F42081318167
:106DB000820F931F2091E6063091E70628173907C6
:106DC00009F061C0F093E706E093E606DF91CF910A
:106DD0000895EA01CE17DF07E8F54A815B819E013D
:106DE00041155105B1F7E901FB83EA8349915991B6
:106DF000C40FD51FEC17FD0761F4808191810296C5
:106E0000840F951FE90199838883828193819B83F5
:106E10008A83F0E0E0E012968D919C9113970097A1
:106E2000B9F52D913C911197CD010296820F931FD8
:106E30002091E6063091E7062817390739F6309792
:106E400051F51092E9061092E806B093E706A09378
:106E5000E606BCCFD383C28340815181840F951F46
:106E6000C817D90761F44E5F5F4F88819981480F39
:106E7000591F518340838A819B819383828321158B
:106E8000310509F0B0CFF093E906E093E8069ECF14
:106E9000FD01DC01C0CF13821282D7CFB0E0A0E0A9
:106EA000E4E5F7E30C94C8328C01009751F4CB0170
:106EB0000E9429368C01C801CDB7DEB7E0E10C9401
:106EC000E432FC01E60FF71F9C0122503109E21762
:106ED000F30708F49DC0D901CD91DC911197C61735
:106EE000D70798F0C530D10530F3CE010497861747
:106EF000970708F3C61BD70B2297C193D1936D93C5
:106F00007C93CF010E94C536D6CF5B01AC1ABD0A77
:106F10004C018C0E9D1EA091E806B091E906512C03
:106F2000412CF12CE12C109731F58091E6069091DF
:106F3000E7068815990509F05CC04616570608F063
:106F400058C08091870190918801009741F48DB7D6
:106F50009EB740918B0150918C01841B950BE817D3
:106F6000F90708F055C0F093E706E093E606F9014B
:106F700071836083A0CF8D919C91119712966C9034
:106F8000129713967C901397A815B90559F56C01C3
:106F900042E0C40ED11CCA14DB0420F1AC014A1932
:106FA0005B09DA011296159780F062827382518331
:106FB0004083D9016D937C93E114F10471F0D70102
:106FC0001396FC93EE93129776CF22968C0F9D1F0B
:106FD000F90191838083F301EFCFF093E906E09309
:106FE000E80669CF4816590608F42C017D01D30143
:106FF0009ACFCB010E9429367C01009749F0AE015F
:10700000B8010E940B38C8010E94C536870153CFD2
:1070100010E000E050CFFB01DC0102C001900D92B6
:1070200041505040D8F70895FB01DC018D9101904B
:1070300080190110D9F3990B0895FB01DC0101902F
:107040000D920020E1F7089510E0C2E6D0E004C000
:10705000FE010E9423362196C336D107C9F7F89462
:02706000FFCF60
:1070620070E9D700640032001F1115111D1D111F98
:107072001F1115111515111F1F111D1D1D1D1D1F7E
:107082001F1117111515111F1F1117111D1D111F8A
:107092001F1515111D1D1D1F1F111D111D1D111F56
:1070A2009600C800FA002C015E019001C201F401B1
:1070B200260258028A02BC02EE0220035203840313
:1070C2009803A203AC03B60370820300F40100002C
:1070D2000500A8FDFFFFB80B000040420F00183D5D
:1070E20087000170E9D7000000EA06800000020470
:1070F2000003000110030200000302010006000465
:1071020000060500200605040000000000E5044515
:107112000472043205A304810495040000000036C1
:10712200070907A507E606EA00F606E706000000DB
:10713200005A0A4504A507360431487A2000313046
:10714200487A003530487A003130304800353030E6
:107152004800316B487A0031306B48003130306B77
:10716200004175746F006E616E00696E66006F7625
:107172006600202050494E204130203D2000302022
:1071820042616C6C203D204F46462056464F2000FF
:10719200332042616C6C3D20302E38206D6B5620BE
:1071A20000362042616C6C3D2036206D6B562020EB
:1071B2002000392042616C6C3D203530206D6B56C9
:1071C200202000392B323064423D20353030206D92
:1071D2006B562000392B343064423D20353030303C
:1071E200206D6B5600392B363064423D20353030ED
:1071F20030306D6B5600535342004F6E20004F6685
:10720200660055004C534200535752202020202044
:1072120020503D30572020202020005357523D005F
:1072220020503D005720202000FFFFFFFFFFFFFFFF
:10723200FF072B363000FFFFFFFFFFFFFFFF072B8B
:10724200353500FFFFFFFFFFFFFFFF072B35300043
:10725200FFFFFFFFFFFFFFFF072B343500FFFFFF9C
:10726200FFFFFFFFFF072B343000FFFFFFFFFFFF91
:10727200FFFF072B333500FFFFFFFFFFFFFFFF0775
:107282002B333000FFFFFFFFFFFFFFFF072B3235DD
:1072920000FFFFFFFFFFFFFFFF072B323000FFFF62
:1072A200FFFFFFFFFFFF072B313500FFFFFFFFFF4F
:1072B200FFFFFF072B313000FFFFFFFFFFFFFFFF44
:1072C200072B352000FFFFFFFFFFFFFFFF072020F6
:1072D2002000FFFFFFFFFFFFFF062020202000FF0E
:1072E200FFFFFFFFFF05202020202000FFFFFFFF00
:1072F200FF0420202020202000FFFFFFFF0320208A
:10730200202020202000FFFFFF022020202020201C
:10731200202000FFFF01202020202020202020000C
:10732200FFFF2020202020202020202000FF2020DE
:10733200202020202020202020002020202020206B
:1073420020202020202000436F72722E504C4C20AF
:1073520053693533353120200020436F72726563E3
:10736200742E2042464F2D32200020202020204320
:107372004C4B202D20322020202000202020434C66
:107382004B31203D3E2056464F2020200020203EFB
:1073920020434C4B2D312020202000436F72722E4F
:1073A20046696C7465722073697A6500487A202098
:1073B2002020200020436F72722E20536869667469
:1073C2002043572000436F72722E20535F4C455664
:1073D200454C2D3F004C00555342004641003B00B6
:00000001FF
